S01F00006F70656E626C745F6F6C696D6578696E6F5F73746D33322E73726563C6
S3150800000000500020950500086D05000871050008D8
S3150800001075050008790500087D0500080000000040
S315080000200000000000000000000000008105000834
S315080000308505000800000000890500088D050008F0
S31508000040DD050008DD050008DD050008DD050008FA
S31508000050DD050008DD050008DD050008DD050008EA
S31508000060DD050008DD050008DD050008DD050008DA
S31508000070DD050008DD050008DD050008DD050008CA
S31508000080DD050008DD050008DD050008DD050008BA
S31508000090DD050008DD050008DD050008DD050008AA
S315080000A0DD050008DD050008DD050008DD0500089A
S315080000B0DD050008DD050008DD050008DD0500088A
S315080000C0DD050008DD050008DD050008DD0500087A
S315080000D0DD050008DD050008DD050008DD0500086A
S315080000E0DD050008DD050008DD0500080000000044
S315080000F000000000000000000000000000000000F2
S3110800010000000000000000005FF808F195
S3150800010C10B5054C237833B9044B13B10448AFF337
S3150800011C00800123237010BD980200200000000007
S3150800012CF46F000808B5034B1BB103490348AFF33A
S3150800013C008008BD000000009C020020F46F000837
S3150800014C03F058BF03F068BF4FF48052024B0128E6
S3150800015C0CBF5A611A61704700100140704700BF06
S3150800016C704700BF08B5054B9B68DB0701D4002018
S3150800017C08BD00F0A5F8012008BD00BF0008014025
S3150800018C642000F06FB800BF00F072B800B5C7B0B5
S3150800019C002168464FF48C7206F010FF6946094830
S315080001AC06F03CFB50B9009828B19DF8080080F081
S315080001BC1000C0F3001047B05DF804FB002047B0F0
S315080001CC5DF804FB1C700008004870471C7000089A
S315080001DC002310B5064C0A222046064984F8283214
S315080001EC05F06CFF10B9012384F8283210BD00BF46
S315080001FCB40200200C70000808B5084890F828329C
S3150800020C012B04D0BDE80840054806F035BB06F0BE
S3150800021C41FABDE80840024806F02EBBB40200209D
S3150800022C1C700008034890F82832012B00D0704740
S3150800023C06F030BAB402002010B5094C94F82832EE
S3150800024C012B00D010BD214606F096FB0028F9DAE2
S3150800025C0023204684F82832BDE8104006F01ABA66
S3150800026CB4020020014B1880704700BFE004002040
S3150800027C10B503F0C5FC0E4C236898420DD30D4BF4
S3150800028C1A785AB1002020210B4A1870516103F0D4
S3150800029CB7FC0A4B1B881844206010BD012020218E
S315080002AC02F1804202F5843218701161EFE700BF43
S315080002BCE4040020E204002000080140E0040020C9
S315080002CC2022014B5A61704700080140244910B599
S315080002DC0A460B6823F0070343F002030B60136806
S315080002EC03F00703022BFAD11E4B1A46196841F480
S315080002FC8031196013689903FCD55168194B21F4A0
S3150800030C7C1141F4E8115160116841F0807111605B
S3150800031C1A689201FCD55A68124C22F0F0025A60FF
S3150800032C5A6822F4E06242F480625A605A6822F4EF
S3150800033C60525A605A6822F0030242F002025A606E
S3150800034C636803F00C03082BFAD1074802F0F8F996
S3150800035C002000F04FF9636823F48003636010BD36
S3150800036C002002400010024000A24A0480B5002476
S3150800037C8AB000F063F9FFF7A9FF4FF0200E0420AE
S3150800038C0827CDE907442E4B4FF4805C9A6940F256
S3150800039C0111012542EA0E029A619A69294E02EA6E
S315080003AC0E020192019A9A69DFF8A09002439A61AB
S315080003BC9A69DFF89C8002400292029A9A693A433B
S315080003CC9A619A693A400392039A9A6942F0100222
S315080003DC9A619B6903F010030493049BC6F814E016
S315080003ECC9F814C0C8F814000591304605A9069733
S315080003FC0995022701F014FA42F2200305A93046A2
S3150800040C059306950894079701F00AFA0E4B05A969
S3150800041C48460593CDE90657089401F001FA40F2CF
S3150800042C0442032305A940460592079306950894AA
S3150800043C01F0F6F9FFF784FEFFF784FEFCE700BF30
S3150800044C0010024000080140100010040010014082
S3150800045C00140140104B82B09969104A41F0010111
S3150800046C9961996901F0010100910099D96941F0E6
S3150800047C8051D961DB6903F080530193019B536862
S3150800048C23F0E06343F080635360536823F0E06322
S3150800049C536002B0704700BF0010024000000140D4
S315080004AC0268094B9A4200D0704703F5DA33DA69C9
S315080004BC82B042F40002DA61DB6903F400030193AB
S315080004CC019B02B0704700BF005C00400268044BF9
S315080004DC9A4204D1034AD36923F40003D3617047C3
S315080004EC005C00400010024008B501F017FA1748E6
S315080004FC01F03EF9164801F03BF9164801F038F9B7
S3150800050C154801F035F9154BDA6922F40002DA615F
S3150800051CDA6922F00072DA619A6922F020029A618D
S3150800052C9A6922F010029A619A6922F008029A6175
S3150800053C9A6922F004029A61DA6922F08052DA6129
S3150800054C9A6922F001029A6108BD00BF00140140A5
S3150800055C00100140000C0140000801400010024048
S3150800056C704700BFFEE700BFFEE700BFFEE700BF0F
S3150800057CFEE700BF704700BF704700BF704700BF5B
S3150800058C00F06EB8704700BF002103E00B4B5B58B8
S3150800059C435004310A480B4B42189A42F6D30A4A7E
S315080005AC02E0002342F8043B084B9A42F9D3FFF7C2
S315080005BCE9FF06F0BFFCFFF7D9FE7047387800084C
S315080005CC000000209402002098020020481B0020FE
S315080005DCFEE7000010B54FF0FF320024044BDA603A
S315080005EC1C61DA60DC60FFF77FFF204610BD00BF98
S315080005FC0010024038B54FF47A730D490D4A097844
S3150800060C1268B3FBF1F30546B2FBF3F000F07CF885
S3150800061C08B90F2D01D9012038BD044602462946D2
S3150800062C4FF0FF3000F03AF8034B20461D6038BDFA
S3150800063C040000200000002008000020074A08B526
S3150800064C1368032043F01003136000F015F800201C
S3150800065CFFF7D0FFFFF7FEFE002008BD0020024082
S3150800066C034A044B11681B780B441360704700BF90
S3150800067CE0180020040000204FF6FF01064A00028D
S3150800068CD36800F4E0600B4043F0BF6343F40033D7
S3150800069C0343D360704700BF00ED00E0184B30B43D
S315080006ACDB68C3F30223C3F10705042D03F1040425
S315080006BC28BF0425062C19D94FF0FF34033B9C4060
S315080006CC22EA04044FF0FF32AA4021EA020101FA99
S315080006DC03F2224312010028D2B20ADB00F1604071
S315080006EC00F5614080F8002330BC7047002423468F
S315080006FCE8E7044B00F00F0003441A7630BC704749
S3150800070C00ED00E0FCEC00E00138B0F1807F0DD282
S3150800071C30B4F02500220721054B064C586084F8A6
S3150800072C2350104630BC9A601960704701207047F8
S3150800073C10E000E000ED00E0124BDB6813F010034C
S3150800074C05D010231049CA6942F00202CA610D4A43
S3150800075CD268500706D50C4943F00403CA6942F01F
S3150800076C0102CA61074AD169C90708D50648C16991
S3150800077C41F00401C161D16921F00101D161014A3D
S3150800078CD360704700200240E8180020064B186911
S3150800079C10F0800006D00549054A59605A60186958
S315080007ACC0F3C010704700BF002002402301674504
S315080007BCAB89EFCD034A0020136943F0800313611C
S315080007CC704700BF0020024070B5054603F026FAB4
S315080007DC134C064601E06A1C12D1E368DB07FAD40F
S315080007ECE368980644BF2023E3600D4BDA68D1060C
S315080007FC02D4DA69D2070BD5FFF79EFF012070BD2C
S3150800080C25B103F00BFA801BA842E6D9032070BD6C
S3150800081CD86810F00400F2D0FFF78EFF0120EEE73F
S3150800082C002002402DE9F04F274E0746307E83B054
S3150800083C012843D09A4601234CF250300D46904677
S3150800084C3376FFF7C1FFA0BB012F3BD0022F0CBF9D
S3150800085C0223042301934FF0000B5F46DFF86C90DC
S3150800086C4FEA0B14C4F12001F7610AFA01F128FAD0
S3150800087C04F2203C0A432AFA04F4D9F8101022434D
S3150800088C92B241F00101C9F810104CF250302A808E
S3150800089CFFF79AFFD9F810200BF1010B22F0010291
S315080008AC5FFA8BF10235C9F8102010B9019B8B42FF
S315080008BCD6D80023337603B0BDE8F08F022003B0F8
S315080008CCBDE8F08F0197C6E7E81800200020024023
S315080008DC2DE9F843DFF8C09099F81830012B56D05B
S315080008EC012203680646022B884689F818204CF222
S315080008FC50302FD0FFF768FF78BB4FF0FF33C8F89E
S3150800090C0030D6E9025305EB83239D4225D20746D0
S3150800091C204C07E0D6E9023205F5806503EB822305
S3150800092CAB421BD9C9F81C7023694CF2503043F002
S3150800093C020323616561236943F040032361FFF7D2
S3150800094C43FF236923F0020323610028E2D0C8F889
S3150800095C005003E0FFF738FF28B10120002389F87F
S3150800096C1830BDE8F8830B4CC9F81C0023694CF207
S3150800097C503043F004032361236943F04003236199
S3150800098CFFF722FF236923F004032361E6E702201D
S3150800099CBDE8F88300200240E8180020F0B587B0BF
S315080009AC002873D090F8A932044603F0FF02002BF6
S315080009BC67D00323254684F8A932206801F022F86B
S315080009CC55F810CB6F462E460FCE0FC73368261D2B
S315080009DC3B60604696E80E0001F002F8074630B117
S315080009EC0223012584F8A932284607B0F0BD014632
S315080009FC206801F011F8606858B339464FF0010CBD
S31508000A0C3A4601EB810304EBC3034F1C83F8281009
S31508000A1CD986F9B2814283F829C083F82B20C3E919
S31508000A2C0E221A64EDD30022114602EB820304EB64
S31508000A3CC303571C83F86821FAB2824283F86911FA
S31508000A4C83F86B11C3F87811C3F87C11C3F88011BD
S31508000A5CEBD30FCD6F46D4F800C00FC72B68604692
S31508000A6C3B6096E80E0000F0D9FF05460028B7D182
S31508000A7C012384F82400206884F8A93201F022FEA8
S31508000A8CB2E780F8A822FFF70BFD92E70125284666
S31508000A9C07B0F0BD38B540B104460323006884F8A6
S31508000AACA93201F0FBFD054610B10125284638BDD3
S31508000ABC2046FFF70BFD84F8A952284638BD00BF1F
S31508000ACC38B590F8A832012B11D0044601250068D8
S31508000ADC84F8A85200F08CFF2946204606F022FA24
S31508000AEC206801F0EDFD002084F8A80238BD02202C
S31508000AFC38BD00BF90F8A832012B12D010B50123CF
S31508000B0C0446006884F8A83200F07CFF00212046D1
S31508000B1C06F008FA206801F0D5FD002084F8A80232
S31508000B2C10BD0220704700BF2DE9F04F044687B070
S31508000B3C006801F0C9FD0304D4F800C000F18B80ED
S31508000B4C604601F0C1FD430500F1A081206801F063
S31508000B5CBBFD10F4804F206807D0B0F8443023F45E
S31508000B6C80431B041B0CA0F8443001F0ADFD10F4B7
S31508000B7C005F206807D0B0F8443023F400531B04F8
S31508000B8C1B0CA0F8443001F09FFDC70400F16081EE
S31508000B9C206801F099FD060546D521680DF1060376
S31508000BAC08460A461D4601F1200732F8046B97429F
S31508000BBC25F8026FF9D1B1F8402042F00102A1F8EC
S31508000BCC4020B1F8402022F001021204120CA1F8C0
S31508000BDC4020B1F844205505FBD5B1F844200DF159
S31508000BEC160522F480621204120CA1F8442033F87C
S31508000BFC022FAB4220F8042BF9D1B1F8403020462D
S31508000C0C43F00803A1F84030B1F8443023F40063EC
S31508000C1C1B041B0CA1F84430B1F8403043F0040314
S31508000C2CA1F8403006F074F8206801F04DFD8205F5
S31508000C3C00F10181206801F047FDC30508D522683B
S31508000C4CB2F8443023F480731B041B0CA2F844300E
S31508000C5C07B0BDE8F08FDFF83C94DFF83CA4DFF86A
S31508000C6C3CB4BCF844301A047FF56AAFBCF844109F
S31508000C7C89B211F00F055BD111F01001BCF80030E8
S31508000C8C00F022819BB213F4006540F057811F04D3
S31508000C9CE7D540F68F73BCF80020134043F0800369
S31508000CACACF80030BCF8503094F8682103EBC2035A
S31508000CBC0CEB4303B3F80C34C3F30903C4F88431BF
S31508000CCCA3B1D4F87C1189B16046B4F86E2101F051
S31508000CDC11FDD4F87C31D4F8842129461344C4F880
S31508000CEC7C31204605F0EEFFD4F800C0BCF8503035
S31508000CFCD4F878219BB20CF20C41002A40F0B5814D
S31508000D0CCA5A22F4F8421204120CCA52CA5A4AEAAD
S31508000D1C020292B2CA52BCF80020DD4B134083F48F
S31508000D2C405343F4004343F08003ACF8003098E793
S31508000D3C3CF82560AF00B6B231043AD4310690D5EA
S31508000D4C3CF8253007EB050809EA030343F400438E
S31508000D5C2CF8253004EBC80898F82B300CF5806E67
S31508000D6C022B00F03E8198F82830D8F84000DB00BA
S31508000D7CBCF85020134402333EF81330C3F309036E
S31508000D8C834280F0CE802F4404EBC707FA6B7E6C47
S31508000D9C0135C01A1A4405EB85053344386404EB4F
S31508000DACC5016046FA637B6401F08AF8D4F800C082
S31508000DBC57E740F68F733CF825207919134043F012
S31508000DCC80032CF8253004EBC10191F874210CF53D
S31508000DDC8063002A40F0D580BCF8502091F8680151
S31508000DEC063202EBC00233F81280C8F30908B8F1D0
S31508000DFC000F40F069817919C9006318D3F884018A
S31508000E0CD3F87C214044C3F88401D3F880014244CA
S31508000E1CC3F87C2120B1D3F87831434540F22F81B1
S31508000E2C7B1904EBC30393F86811204605F04AFFB7
S31508000E3CD4F800C082E722682046B2F8443023F47E
S31508000E4C00731B041B0CA2F8443005F04FFFF1E6A7
S31508000E5C22682046B2F8403023F004031B041B0C0E
S31508000E6CA2F84030B2F8403023F008031B041B0CE0
S31508000E7CA2F8403005F05EFF2068B0F8443023F441
S31508000E8C80531B041B0CA0F8443082E622682046CB
S31508000E9CB2F8443023F480631B041B0CA2F84430CC
S31508000EAC05F028FF94F8A832012B3FF44FAE002525
S31508000EBC012384F8245084F8A8322946206801F0C6
S31508000ECCF9FB84F8A85241E609EA030343F4004304
S31508000EDCACF80030BCF8503094F82800E26B03EB01
S31508000EECC0030CEB430CBCF804342046C3F30903CB
S31508000EFC1A446364E26305F0EFFE94F82430002B81
S31508000F0C3FF454AF236CD4F800C0002B7FF4A9AE81
S31508000F1C94F8242042F08002ACF84C2084F8243053
S31508000F2C9FE600233D4404EBC5052B6498F828106E
S31508000F3C204605F0D1FED4F800C092E6BCF8503035
S31508000F4C94F86821604603EBC2030CEB430CBCF81F
S31508000F5C0C34B4F86E21C3F30903C4F8843104F5D0
S31508000F6C2C7101F0C7FB40F68F7322682046118856
S31508000F7C0B4043F08003138005F09EFED4F800C0A6
S31508000F8C6FE691F86B0191F86821022800F0D18080
S31508000F9C3CF8220020F0F0000005000D40F400405B
S31508000FAC40F0C0002CF8220091F868213CF8220089
S31508000FBC10F4804FBCF8500072D0023000EBC2021D
S31508000FCC33F81280C8F30908B8F1000F3FF413AFD1
S31508000FDCB1F8702160464346D1F87C1101F08AFBC2
S31508000FEC09E798F82810F205D8F840004FEAC1032B
S31508000FFC7FF5BEAE06F4804216F040060196BCF8A4
S3150800100C5060334473D106333EF81330C3F30903E7
S3150800101C834200F24D81C01AC8F84000002800F03F
S3150800102C4A815AB93CF8212022F0F0021205120D19
S3150800103C42F4404242F080022CF821207A1904EB43
S3150800104CC20292F84C10012900F0608198F8282009
S3150800105C3CF822300BEA030383F0300343F40043D5
S3150800106C43F080032CF82230FBE53E2A35D850088D
S3150800107CD60748BF0130820292B2CA524BE601F536
S3150800108CB4712144206800F01BFFD4F800C055E663
S3150800109C8FBFFFFF0F8FFFFF0080FFFFBF8FFFFF84
S315080010AC063000EBC20233F81280C8F30908B8F10F
S315080010BC000F3FF4A0AEB1F8722160464346D1F852
S315080010CC7C1101F017FB96E6B1F86E216046434693
S315080010DCD1F87C1101F00EFB8DE65009D50608BF38
S315080010EC00F1FF304AEA802292B2CA5213E6023362
S315080010FC3EF81330C3F30903834257D30023204623
S3150800110CC8F84030019205F0E7FD019AD4F800C002
S3150800111C002A9BD098F828203CF8223023F0F003BC
S3150800112C1B051B0D43F4404343F080032CF8223077
S3150800113C8CE716F48040BCF8508001904FEAC20048
S3150800114CD1F880E1404400F08580023033F8103045
S3150800115CC3F309037345984600F2C880AEEB030047
S3150800116CC1F88001002800F0C480720610D57A19DF
S3150800117C04EBC20292F868113CF8212022F0F00226
S3150800118C1205120D42F4004242F0C0022CF821203E
S3150800119C0BB998462FE6791904EBC101B1F8702101
S315080011AC6046D1F87C1101F0A5FA24E6C01AC8F8F5
S315080011BC40005AB13CF8212022F0F0021205120D1B
S315080011CC42F4404242F080022CF821207A1904EBB2
S315080011DCC20292F84C1001297FF438AFD2E91116E5
S315080011ECD06BD2F838E0184419447645D06351646C
S315080011FCC0F0D480A6EB0E06966498F829201FFA40
S3150800120C8EF31E46002A40F0BB8098F82820BCF8BE
S3150800121C50100CEB021202F2044289B25318BEF1BA
S3150800122C000F40F0E6807346565A26F4F846360404
S3150800123C360C5652565A4AEA0606B6B256527A1917
S3150800124C04EBC2020146128E604601F043FAD4F84A
S3150800125C00C0FBE6063033F81030C3F309037345B8
S3150800126C984633D8AEEB0300C1F8800188B37006F4
S3150800127C10D47A1904EBC20292F868113CF82120B2
S3150800128C22F0F0021205120D42F4004242F0C0029E
S3150800129C2CF82120002B3FF47CAF791904EBC10103
S315080012ACB1F872216046D1F87C1101F023FAA2E557
S315080012BC019BC8F840302046019205F00DFD019AB5
S315080012CCD4F800C0002A3FF425AFBFE60198C1F850
S315080012DC80013CF822006B49014081F4005141F42D
S315080012EC004141F080012CF82210C0E70020C1F81B
S315080012FC80013CF822006349014081F4005141F415
S3150800130C004141F080012CF822102EE7D06BD2F860
S3150800131C38E0D2E91116184419447645D06351645D
S3150800132C4FD3A6EB0E06966498F829201FFA8EF36F
S3150800133C1E46002A38D198F82820BCF850100CEB19
S3150800134C021202F20C4289B25318BEF1000F71D187
S3150800135C7346565A26F4F8463604360C5652565ADE
S3150800136C4AEA0606B6B256527A1904EBC202014686
S3150800137C528E604601F0AEF9D4F800C066E6B3B2F8
S3150800138C012A7FF45CAF98F82820BCF850100CEBB7
S3150800139C021202F2044289B2535250E7B6B982F8E5
S315080013AC4C609E4629E7B3B2012ADDD198F828206D
S315080013BCBCF850100CEB021202F20C4289B25352D2
S315080013CCD2E726BB82F84C609E46ADE7002382F82E
S315080013DC4C30936498F82920002AD0D198F82830F4
S315080013ECBCF850200CEB031303F20443B646134423
S315080013FCB6B2BEF13E0F2BD84FEA5E021EF0010FB5
S3150800140C18BF0132920292B21A80334617E70023AC
S3150800141C936482F84C3098F82920002AC3D198F89E
S3150800142C2830BCF850200CEB031303F20C43B646D9
S3150800143C1344B6B2BEF13E0F17D84FEA5E021EF041
S3150800144C010F18BF0132920292B21A8033468BE70B
S3150800145C4FEA5E121EF01F0F08BF02F1FF324AEA6E
S3150800146C822292B21A803346E9E64FEA5E121EF0E1
S3150800147C1F0F08BF02F1FF324AEA822292B21A8083
S3150800148C334671E78FBFFFFF90F8A832012B0DD0BA
S3150800149C012110B5044680F8A81205F043FD206812
S315080014AC01F00EF9002084F8A80210BD022070473E
S315080014BC90F8A832012B0ED0012310B5044680F8FB
S315080014CCA832002105F02EFD206801F0FBF800205B
S315080014DC84F8A80210BD0220704700BF90F8A82215
S315080014EC012A0DD010B50446012284F8241080F880
S315080014FCA822006801F0DEF8002084F8A80210BDC6
S3150800150C0220704770B501F00705090622D400269B
S3150800151C05EB8504E40004F5B4710444014484F82D
S3150800152C69614C780D700A61CB7004B1CD81022BC0
S3150800153C04BF00230B7190F8A832012B12D001239B
S3150800154C044680F8A832006800F07CFA002084F87B
S3150800155CA80270BD0124291901EB810100EBC10118
S3150800156C4C70DEE7022070BD0B0610B501F00702C1
S3150800157C19D4002402EB8203DB0003F5B471014491
S3150800158C034483F869410A7090F8A832012B16D0E7
S3150800159C0123044680F8A832006800F0BBFB002043
S315080015AC84F8A80210BD0123D11801EB810100EBC8
S315080015BCC1010A704B7090F8A832012BE8D10220B1
S315080015CC10BD00BF70B5002601F0070101EB8104C0
S315080015DCE400051904F5B47485F86811C5F87C217E
S315080015EC0119C5F880310068C5F8846185F8696108
S315080015FC00F066FC304670BD01F0070101EB810175
S3150800160C00EBC101D1F88401704700BF70B5012603
S3150800161C002501F0070101EB810400EBC404E26329
S3150800162C8A1902EB820284F82810236400EBC201A3
S3150800163CA364006884F84C6084F82960656400F03B
S3150800164C3FFC284670BD00BF38B5436801F0070556
S3150800165C9D421DD80B061DD4002401EB8101C9003F
S3150800166C431883F86941012301F5B47281180D708A
S3150800167C8B7090F8A8229A421AD0044680F8A832A1
S3150800168C006800F095FFADB1002084F8A80238BDBB
S3150800169C012038BD0123E91801EB810100EBC101DA
S315080016AC4B7001230D708B7090F8A8229A42E4D1E6
S315080016BC022038BD04F52C71206801F009F8E3E71F
S315080016CC38B5436801F00F029A421FD80B0601F091
S315080016DC07021DD40024002502EB8203DB0003F568
S315080016ECB4710144034483F869410A708D7090F80B
S315080016FCA832012B1AD00123044680F8A8320068B8
S3150800170C00F078FF84F8A852284638BD012038BD69
S3150800171C01230025D11801EB810100EBC1010A70E8
S3150800172C8D704B7090F8A832012BE4D1022038BD8D
S3150800173C11F0800F0FD001F00701013101EB810187
S3150800174C00EBC10198B27AB101221B0C08814B81BE
S3150800175C0A730020704701EB810100EBC10101F50A
S3150800176CB47198B2002AEFD1C8800A73002070476A
S3150800177C264B98420DD0264B98422ED0254B984294
S3150800178C13D0254B984234D0244B984219D00120BB
S3150800179C704703F58433DA68002042F00402DA60F5
S315080017ACDA6822F00402DA60704703F58033DA68E7
S315080017BC002042F01002DA60DA6822F01002DA60D1
S315080017CC704703F57843DA68002042F04002DA6085
S315080017DCDA6822F04002DA60704703F58233DA6879
S315080017EC002042F00802DA60DA6822F00802DA60B1
S315080017FC704703F57C43DA68002042F02002DA6071
S3150800180CDA6822F02002DA60704700BF000801404F
S3150800181C000C014000100140001401400018014062
S3150800182C2DE9F0470F68C7F30F2797FAA7F6B6FA0C
S3150800183C86F637FA06F36ED04FF0010C4FF00F0E02
S3150800184C4FF003084FF0040A56E040F20113B34078
S3150800185CC2684FEA132999FAA9F4B4FA84F50C6903
S3150800186C22EA0902AC402243C2601C0E93FAA3F585
S3150800187CB5FA85F593FAA3F2B2FA82F2AD004FEAFD
S3150800188C820902590EFA05F522EA05054A6802FA92
S3150800189C09F2154305514A6822F00802012A27D194
S315080018AC93FAA3F2B2FA82F293FAA3F9B9FA89F97E
S315080018BC920008FA02F225EA02058A684FEA8909B3
S315080018CC02FA09F22A43025193FAA3F9B9FA89F9E9
S315080018DC93FAA3F3B3FA83F3CD684FEA89099B000D
S315080018EC0AFA09F922EA090205FA03F31343035122
S315080018FC013637FA06F30ED00CFA06F33B42F7D04C
S3150800190C072EA2D94FF00112A6F1080302FA03F327
S3150800191C43F080639CE70020BDE8F087164B1A4617
S3150800192C196841F00101196013689B07FCD55368C7
S3150800193C114923F0030353604B6813F00C0FFBD1CA
S3150800194C0B680D4A23F080730B60136813F0007351
S3150800195CFBD153601168184621F4502111601168A7
S3150800196C21F0F80141F0800111609360536A43F04D
S3150800197C80735362704700BF00100240026812F071
S3150800198C40022AD1F0B4D1E90035044688682B43C5
S3150800199CCD68034308692B434D698E690343CF69A8
S315080019AC20682B4333430E6A3B4320F47F40334372
S315080019BC20F0BF00034323606368B6F5005F23F08D
S315080019CC040343EA1543636002D0F0BC1046704723
S315080019DC8B8C10462361F0BC70470120704700BF02
S315080019EC84B001A880E80E0004B00020704700BF40
S315080019FC03464FF43F420020A3F84400A3F84020C6
S31508001A0C704700BF44F2FF030246B0F840100020AE
S31508001A1C0B40A2F8403070470020704784B030B4B1
S31508001A2C044601200025A4F8400003A8A4F8405059
S31508001A3C80E80E00A4F844502846A4F8505030BC50
S31508001A4C04B0704770B40D78034630F82540AC4A9C
S31508001A5CC8782240032800F22481DFE800F04E46BD
S31508001A6C024A002048F28004224323F825200D78E8
S31508001A7CA44E33F825202C433240224323F8252044
S31508001A8C0A7B002A3DD1CC880A784D786408640014
S31508001A9C03EB0212002D00F0CA80B3F850502A440A
S31508001AACA2F800440A7833F8225003EB82046D0638
S31508001ABC0BD533F82240264046F4004646F0C006BD
S31508001ACC23F822600C7803EB8404CB78012B00F006
S31508001ADC008122888C4B134083F0200343F4004387
S31508001AEC43F08003238070BC704742F48062002068
S31508001AFCB8E742F4C0620020B4E742F40072002052
S31508001B0CB0E70C7833F82420324042F4014242F014
S31508001B1C800223F824200A780C89B3F8505003EB7A
S31508001B2C0212640802F580626400ADB254530A7856
S31508001B3C4C89B3F8505003EB0212640802F5816223
S31508001B4C6400ADB254530C784A7833F8245092BBDF
S31508001B5C6D0403EB84020BD533F82420164046F4A7
S31508001B6C404646F0800623F824600A7803EB820286
S31508001B7C148866060CD5148824F0F0042405240D64
S31508001B8C44F4004444F0C00414800A7803EB82023F
S31508001B9C48F2800516885D4C344084F440542C4336
S31508001BAC14800978584A33F821402240154323F803
S31508001BBC215070BC70476D0403EB84020BD533F8C7
S31508001BCC2420164046F4404646F0800623F8246046
S31508001BDC0A7803EB8202148864060CD5148824F060
S31508001BECF0042405240D44F4004444F0C004148085
S31508001BFC0A7803EB8202CC78012C5FD01588424C0C
S31508001C0C2C4084F0200444F4004444F080041480EE
S31508001C1C097870BC33F8212022F0F0029204920C59
S31508001C2C42F4004242F0800223F821207047B3F8B0
S31508001C3C50600D693244A2F808440A78B3F850404B
S31508001C4C03EB021202F20C42A4B265B33E2D4BD83A
S31508001C5C6E08ED0748BF0136B602B6B216530C78B5
S31508001C6C33F8245003EB84026E040ED533F8242083
S31508001C7C22F0F0021205120D42F4404242F08002A4
S31508001C8C23F824200A7803EB820211881F4B70BCB8
S31508001C9C0B4083F4405343F4004343F08003138012
S31508001CAC70470120DEE6155B25F4F8452D042D0C4E
S31508001CBC1553155B45F400451553D0E7148824F0E5
S31508001CCCC0042405240D44F4004444F08004148014
S31508001CDC9EE7238823F0C0031B051B0D43F4004322
S31508001CEC43F08003238064E76E09ED06084D08BFB0
S31508001CFC06F1FF3645EA8625ADB21553AFE700BFA8
S31508001D0C8F89FFFF8F8FFFFFBF8FFFFF8FBFFFFFEF
S31508001D1C0080FFFF30B40A780D7B00EB82034C7809
S31508001D2C15BB002C00F0998030F8224064060ED5BD
S31508001D3C30F8223023F0F0031B051B0D43F4004347
S31508001D4C43F0C00320F822300B7800EB83031A8883
S31508001D5C002030BC22F0C0021205120D42F40042DB
S31508001D6C42F080021A807047002C41D130F822408C
S31508001D7C64040ED530F8223023F0F0031B051B0D36
S31508001D8C43F4404343F0800320F822300B7800EBF1
S31508001D9C83031A8855060CD51A8822F0F002120508
S31508001DAC120D42F4004242F0C0021A800B7800EB86
S31508001DBC830348F280051A883F4C22F0F00212057C
S31508001DCC120D42F4004242F0C0021A800A7830F82A
S31508001DDC223023402B4320F822300A78374B30F830
S31508001DEC22100B401D4320F82250002030BC7047AF
S31508001DFC30F8224064040ED530F8223023F0F00374
S31508001E0C1B051B0D43F4404343F0800320F8223096
S31508001E1C0B7800EB83031A8852063ED448F28005E9
S31508001E2C1A88264C22F0F0021205120D42F4404292
S31508001E3C42F080021A800A7830F8223023402B436D
S31508001E4C20F822300A781C4B30F822100B401D4320
S31508001E5C20F82250002030BC704730F82240650428
S31508001E6C0ED530F8223023F0F0031B051B0D43F476
S31508001E7C404343F0800320F822300B7800EB8303B1
S31508001E8C1A88002030BC22F0F0029204920C42F41C
S31508001E9C004242F080021A8070471A8822F0F0023B
S31508001EAC1205120D42F4004242F0C0021A800B7859
S31508001EBC00EB8303B2E700BF8FBFFFFFBF8FFFFFA7
S31508001ECCF0B54B780A7B012B34D042B1CA78022A7A
S31508001EDC00F0DB80012A00F0A7800120F0BD8C6998
S31508001EEC0B6900F20C459C4293BF2346E41A8C619D
S31508001EFC8A610C78B0F8502024012A44002B00F093
S31508001F0C85803E2B00F205815D08DB0748BF01354D
S31508001F1CAD02ADB2A5520A7800EB82021188C14B0C
S31508001F2C00200B4083F4405343F4004343F08003F2
S31508001F3C1380F0BD0F69D1E90534BC4228BF3C4675
S31508001F4C002A3AD0CD780A78022D00F0F08030F8C5
S31508001F5C2250A6B26D064FEA0212B0F8507040F144
S31508001F6C678100F20C453D44AE524D89A2B201324E
S31508001F7C00F58064520804EB450407D004EB820292
S31508001F8C33F8025B24F8045BA242F9D10C784B783F
S31508001F9C00EB8402002B40F0358130F8243023F016
S31508001FACF0031B051B0D43F4004343F0C00320F854
S31508001FBC24300A7800EB82021CE0A5B2CE880135E3
S31508001FCC00F580626D08A4B202EB460207D002EB5C
S31508001FDC850533F8026B22F8046BAA42F9D1B0F8DE
S31508001FEC50500A7800F2044312012B44D4520A7852
S31508001FFC00EB820211888C4B00200B4083F03003D7
S3150800200C43F4004343F080031380F0BDA35A23F432
S3150800201CF8431B041B0CA352A35A43F40043A352C4
S3150800202C0A7800EB820279E78A690D69AA4200F2FE
S3150800203C0581002415468C610A781BBBB0F8503014
S3150800204C00F2044412011C44002D40F07181A35A7D
S3150800205C764E23F4F8431B041B0CA352A35A43F4E1
S3150800206C0043A3524B78002B00F04D81012B0A78C4
S3150800207C08D1B0F8506000F20C441201ABB23444EB
S3150800208CA3520A7800EB820248E70C781BBBB0F81F
S3150800209C50200D6900F2044324011344002D00F06E
S315080020ACF8803E2D00F217816A08EE0748BF013208
S315080020BC920292B21A534B78002B00F01A81012B1C
S315080020CC0C7808D1B0F8506000F20C422401ABB27F
S315080020DC324413530C78CB69A5004219002B3FF4F4
S315080020EC1DAF44F2400630F824303340B34202D0D8
S315080020FC002B7FF413AF435B23F0F0031B051B0D7A
S3150800210C43F4004343F0C00343530A7800EB8202BE
S3150800211C04E75D09DF06454B08BF05F1FF3543EAC1
S3150800212C85239BB2A3520A7800EB8202F6E60D6A67
S3150800213CAF4280F0868030F822602D1B26F4F876A4
S3150800214C3605360D46F4014646F0800620F8226020
S3150800215C0A780D6230F8226016F0400F4E7800F0BF
S3150800216C0081002E40F05881B0F850C000F20C46A1
S3150800217C12016644002C40F0C28136F802C02CF4D9
S3150800218CF84C4FEA0C4C4FEA1C4C26F802C036F8B1
S3150800219C02C04CF4004C26F802C02344AF424B61F3
S315080021AC80F05C812D1B0D624A78002A40F068810C
S315080021BCB0F850200D7800F2044632442D01002C5C
S315080021CC00F050813E2C00F2DA816608E70748BF1A
S315080021DC0136B602B6B2AE52A4B20D89013400F578
S315080021EC8062640802EB450218BF03EB440405D071
S315080021FC33F8025B9C4222F8045BF9D10A7800EBAF
S3150800220C8202F7E6012B7FF4F5AE30F8243023F082
S3150800221CF0031B051B0D43F4404343F0800320F8E1
S3150800222C2430EBE78FBFFFFFBF8FFFFF0080FFFF58
S3150800223C00F204453D44AE520D8997E6521B8A615D
S3150800224CFAE630F8224000F2044624F4F874240521
S3150800225C240D44F4004444F0800420F8224032460D
S3150800226CB0F850700C78AEB23A442401A6523246F5
S3150800227C0D89013200F58064520804EB4504BDD083
S3150800228C03EB420233F8025B934224F8045BF9D160
S3150800229CB4E71A5BC54E22F4F8421204120C1A5310
S315080022AC1A5B42F400421A534B78002B7FF407AFA3
S315080022BCB0F850300A7800F20C441C441201A35AA8
S315080022CC23F4F8431B041B0CA352A35A33439BB2A7
S315080022DCA3520C78FFE66E09EA06B44A08BF06F163
S315080022ECFF3642EA862292B21A534B78002B7FF4B9
S315080022FCE6AEB0F850500B7800F20C442C441B0197
S3150800230CE2520C78E7E6B0F850300A7800F20C4442
S3150800231C12011C44A35A23F4F8431B041B0CA352A6
S3150800232CA35A33439BB2A3520A7800EB8202F5E513
S3150800233C3E2D63D86B08EF0748BF01339B029EB24C
S3150800234CA6524B78002B7FF491AEB0F850400B7820
S3150800235C00F20C4222441B01D6520A7800EB820288
S3150800236CDCE5002E40F0A980B0F850C000F2044617
S3150800237C12016644002C40F0D28036F802C02CF4C8
S3150800238CF84C4FEA0C4C4FEA1C4C26F802C036F8AF
S3150800239C02C04CF4004C26F802C02344AF424B61F1
S315080023AC80F087802D1B0D624A78002A75D1B0F80B
S315080023BC50200D7800F20C4632442D01002C51D0D9
S315080023CC3E2C00F2E7806608E70748BF0136B602DE
S315080023DCB6B2AE52A4B24D89013400F5806202EB56
S315080023EC4502640818BF02EB84043FF407AF33F8C0
S315080023FC025B22F8045BA242F9D1FFE66B09EE06F2
S3150800240C6A4E08BF03F1FF3346EA8326B6B2A652D4
S3150800241C4B78002B99D029E6012E09D1B0F850C07B
S3150800242C00F20C46664412011FFA84FC26F802C018
S3150800243CB1F80AC0A2B2013200F5806606EB4C066A
S3150800244C5FEA520C3FF4A9AE1A4603EB4C0C32F871
S3150800245C02EB944526F804EBF9D19EE600222C46AD
S3150800246C0A62A1E6AB5A23F4F8431B041B0CAB52C5
S3150800247CAB5A43F40043AB520A7800EB8202B9E537
S3150800248C012A7FF4A9AEB0F850600D7800F2044228
S3150800249C32442D01A6B2AE529EE6012A9AD1B0F864
S315080024AC50600D7800F20C4232442D01A6B2AE52A1
S315080024BC90E700222C460A6276E7012E09D1B0F87D
S315080024CC50C000F20446664412011FFA84FC26F832
S315080024DC02C0B1F808C0A2B2013200F5806606EB5C
S315080024EC4C065FEA520C3FF458AF1A4603EB4C0CF9
S315080024FC32F802EB624526F804EBF9D14DE73E2C8F
S3150800250C1DD84FEA540C14F0010F18BF0CF1010C2E
S3150800251C4FEA8C2C1FFA8CFC26F802C088E73E2C56
S3150800252C1DD84FEA540C14F0010F18BF0CF1010C0E
S3150800253C4FEA8C2C1FFA8CFC26F802C0C9E74FEA26
S3150800254C541E14F01F0FDFF864C008BF0EF1FF3ECF
S3150800255C4CEA8E2C1FFA8CFC26F802C068E74FEA68
S3150800256C541E14F01F0FDFF844C008BF0EF1FF3ECF
S3150800257C4CEA8E2C1FFA8CFC26F802C0A9E76709D0
S3150800258CE6060A4E08BF07F1FF3746EA8726B6B2B3
S3150800259CAE5221E66709E606044E08BF07F1FF3777
S315080025AC46EA8726B6B2AE5214E700BF0080FFFF94
S315080025BC4B780A7830F822105BB90C4B0B4083F435
S315080025CC805343F4004343F0800320F82230002064
S315080025DC7047074B0B4083F0100343F4004343F05A
S315080025EC800320F822300020704700BF8FBFFFFF02
S315080025FCBF8FFFFF0B7B002B39D110B40B784C78AF
S3150800260C00EB830214B330F8232052060BD530F8AE
S3150800261C232022F0F0021205120D42F4004242F079
S3150800262CC00220F82320CB78012B1DD00A78194B31
S3150800263C30F8221010BC0B4083F0200343F40043FF
S3150800264C43F0800320F822300020704730F82340EE
S3150800265C64040ED41188104B0B4083F4405343F496
S3150800266C004343F080031380002010BC7047002001
S3150800267C704730F8232022F0F0021205120D42F4AE
S3150800268C404242F0800220F823200A7800EB8202AE
S3150800269CE0E700BFBF8FFFFF8FBFFFFF0346002297
S315080026AC01200321A3F84000A3F844201046A3F800
S315080026BC4010704711B98023A0F84C3000207047A1
S315080026CC0020704700207047B0F84400704700BFE0
S315080026DC00207047013300EB42025B0802F580626A
S315080026EC07D002EB830331F8020B22F8040B9A424B
S315080026FCF9D1704700EB4202580802F580621AD0ED
S3150800270CF0B4174606468D1C37F8044B013EA4B2A6
S3150800271C4FEA142C05F8024C05F801CC05F1020514
S3150800272CF2D1F0BC01EB400102EB8002D80744BFA2
S3150800273C13880B707047DB0744BF13880B70704700
S3150800274C014B1860704700BF0000002070B50B4D98
S3150800275C287301F055FA00F1320605E001F0C0FCC9
S3150800276C01F04EFAB04206D8AC6814F00104F5D064
S3150800277CE868C0B270BD204670BD00BF0038004086
S3150800278C38B501F03DFA00F5FA7503E001F038FAB0
S3150800279CA84209D2FF20FFF7D9FF044601F0A0FC96
S315080027ACFF2CF3D1012038BD002038BD70B50426A6
S315080027BC084DFF206E61FFF7C9FFFFF7E1FF10B167
S315080027CC0124204670BD04462E61FF20FFF7BEFF8C
S315080027DC204670BD0014014070B50E46010604462D
S315080027EC40D40422244BFF201A61FFF7AFFFFFF7F2
S315080027FCDDFFC0B144F04000FFF7A8FF300EFFF72D
S3150800280CA5FFC6F30740FFF7A1FFC6F30720FFF79E
S3150800281C9DFFF0B2FFF79AFF44B1082C19D1872017
S3150800282CFFF794FF05E0FF25284670BD9520FFF7B6
S3150800283C8DFF0A24FF20FFF789FF054601F050FC9F
S3150800284C2A0604F1FF33EFD513F0FF04F2D128461C
S3150800285C70BD0120FFF77AFF0C2CEAD1FF20FFF799
S3150800286C75FFE6E700213720FFF7B6FF0128054676
S3150800287CDAD804F07F04B4E70014014038B5841C98
S3150800288C00F2022514F8020CFFF760FF023414F864
S3150800289C030CFFF75BFFAC42F4D1FF20FFF756FFA2
S315080028ACFF20FFF753FFFF20FFF750FF00F01F0034
S315080028BCA0F10500B0FA80F0400938BDF8B5054618
S315080028CC0E4601F09DF900F1640703E001F098F952
S315080028DCB84222D2FF20FFF739FF044601F000FC6C
S315080028ECFF2CF3D0FE2C18D10235FF20FFF72EFF54
S315080028FC05F8020CFF20FFF729FF05F8010C01F07B
S3150800290CEFFB023E05F10205EFD1FF20FFF71EFF94
S3150800291CFF20FFF71BFF0120F8BD0020F8BD00BF04
S3150800292C60B92DE9F04FB34F99B03D7815F0020513
S3150800293C06D03878C0B219B0BDE8F08F01207047C0
S3150800294C40F204444FF0010B4FF0020AAA4BAB4E6F
S3150800295C9A69304642F008029A619A6904A902F00B
S3150800296C08020192019A9A694FF0040842F0200273
S3150800297C9A619A69DFF8989202F020020292029AFA
S3150800298CDA6942F48042DA61DB69CDE9044B03F477
S3150800299C80430393039B0795CDF818A0FEF740FFD9
S315080029AC09200322964BC6F8108004A905904846C0
S315080029BC069204930795FEF733FF924B04A94846F3
S315080029CCCDE90438FEF72CFF38224FF482704FF409
S315080029DC007107238C4C0F90139120460DEB0201C6
S315080029EC149217930E95CDE910551295CDE91555F8
S315080029FCFEF7C4FF2368854A43F040032360484624
S31508002A0CC6F8108009A9CDE90ABA0C950992FEF701
S31508002A1C07FF4FF400430A264FF0FF08C9F8103099
S31508002A2C01F0EEF800F1640503E001F0E9F88542DF
S31508002A3C02D3A3689907F8D584F80C8001F0E0F85E
S31508002A4C00F1640503E001F0DBF8854202D3A368C4
S31508002A5CDA07F8D5013EE3D1092103224FF0040821
S31508002A6C6A4B664D0A916A4809A90B9209930C960A
S31508002A7CFEF7D6FEC5F8148031463046FFF7ACFE95
S31508002A8C012804460FD0634BFF201E60C5F8108042
S31508002A9CFFF75CFE3B7843F001033B703878C0B215
S31508002AAC19B0BDE8F08F01F0ABF84FF4D57100F50D
S31508002ABC7A780820FFF790FE012817D109AC25462D
S31508002ACC0AAEFF20FFF742FE05F8010BB542F8D116
S31508002ADC9DF82630012B55D0002004224D49474B32
S31508002AEC08601A61FF20FFF731FED3E73146A920AB
S31508002AFCFFF772FE02283ABFA9240225012506E033
S31508002B0C00212046FFF768FE28B101F0E9FA01F02A
S31508002B1C77F84045F4D301F073F84045DCD24FF40E
S31508002B2C00711020FFF758FE0028D5D10422394928
S31508002B3C324B0D60FF201A61FFF708FE00234FF495
S31508002B4C827E4FF4007C082607253A782E4C02F034
S31508002B5CFE023A7022680EA922F040022260204634
S31508002B6C0E93CDE910331293CDE91533CDF83CE02D
S31508002B7CCDE913C61795FEF701FF236843F040030A
S31508002B8C2360D6E69DF82730AA2BA5D105E04FF091
S31508002B9C8041A920FFF720FE18B101F031F8404515
S31508002BACF5D301F02DF8404596D200213A20FFF7CF
S31508002BBC13FE002890D1FF20FFF7C8FD04F8010B7F
S31508002BCCAC42F8D19DF824305B0609D50C200422BA
S31508002BDC10490A4B08601A61FF20FFF7B7FDADE7ED
S31508002BEC04230C49054A0B60FF201361FFF7AEFD61
S31508002BFCA4E700BF0C00002000100240001401409E
S31508002C0CA000A00440004004003800408000800466
S31508002C1C000C0140E804002018B9034B1878C0B220
S31508002C2C70470120704700BF0C00002038B5D8B992
S31508002C3C1C46CBB1204B1B78D8072BD41F4B0D4603
S31508002C4C1B681B0758BF5202012C114625D01220AF
S31508002C5CFFF7C2FD78B101240422194BFF201A6133
S31508002C6CFFF774FD204638BD0424204638BD01F014
S31508002C7C37FA013C09D028464FF40071FFF71EFEBF
S31508002C8C05F500750028F2D1012400210C20FFF768
S31508002C9CA3FDE1E70324204638BD1120FFF79CFD70
S31508002CAC0028D9D128464FF40071FFF707FEB0FA71
S31508002CBC80F46409D0E700BF0C000020E80400206B
S31508002CCC0014014030B583B010BB1C4603B3324B1D
S31508002CDC0D461978C9073CD41B7858073DD42F4B99
S31508002CEC1B68190758BF5202012C41D013F0060F66
S31508002CFC37D111461920FFF76FFDD0B101240422F4
S31508002D0C274BFF201A61FFF721FD204603B030BD83
S31508002D1C0424204603B030BDFC20FFF717FD2846D7
S31508002D2CFFF7ACFD05F5007538B101F0D9F9013C92
S31508002D3C03D0FFF725FD0028EED1FFF721FD00286B
S31508002D4CDCD000344FF0FD0018BF0124FFF7FEFC61
S31508002D5CD5E70324204603B030BD0224204603B031
S31508002D6C30BD214697200192FFF736FD019AC0E740
S31508002D7C11461820FFF730FD0028BFD1FFF700FDDC
S31508002D8C0028BBD0FE20FFF7E1FC2846FFF776FDAE
S31508002D9CB0FA80F46409B2E70C000020E8040020BD
S31508002DAC0014014070B584B0A8B9834B1B78D807BA
S31508002DBC0DD415460E2900F2AA80DFE801F07F4DE6
S31508002DCCA82AA8A8A8A8A8A89B8DA0171000032411
S31508002DDC204604B070BD0424204604B070BD774B61
S31508002DEC1B685B0700F1B88001246CE000213A20CF
S31508002DFCFFF7F2FC0028F7D16C1E0335FF20FFF70E
S31508002E0CA5FC04F8010F01F06BF9A542F6D10024D4
S31508002E1C59E06A4E316811F004017AD000218D20F0
S31508002E2CFFF7DAFC0028DFD1FF20FFF78FFC102113
S31508002E3C6846FFF743FD0028D6D03024FF20013C16
S31508002E4CFFF784FC14F0FF04F8D110239DF80A2030
S31508002E5C120993402B6036E000210920FFF7BCFCD1
S31508002E6C04460028C0D110216846FFF727FD002824
S31508002E7CBAD09DF800309B09012B7FD09DF80730FE
S31508002E8C9DF808609DF806009DF805209DF8091028
S31508002E9C9B0003EB96139DF80A60800202F00F0262
S31508002EAC490000F4406002EBD61201F00601034417
S31508002EBC0A440133073A93402B6004E0FFF776FC8B
S31508002ECCB0FA80F4640904223D4BFF201A61FFF71F
S31508002EDC3DFC204604B070BD00210920FFF77CFCA0
S31508002EEC002881D128461021FFF7E8FCB0FA80F4B7
S31508002EFC6409E8E7314B00241B681370E3E70021EB
S31508002F0C0A20FFF769FC00287FF46EAFEAE7042471
S31508002F1CD9E70920FFF760FC044600287FF464AF64
S31508002F2C10216846FFF7CAFC00283FF45DAF3268EB
S31508002F3C9DF80A3012F002029DF80B002ED05B00A9
S31508002F4C9DF80D2003F07E0303EBD0139209013391
S31508002F5C013A93402B60B6E700218D20FFF73CFC25
S31508002F6C00287FF441AFFF20FFF7F0FB28464021ED
S31508002F7CFFF7A4FCB0FA80F46409A4E79DF80720CF
S31508002F8C9DF8081012049DF8093002F47C120132DF
S31508002F9C03EB012313449B022B6094E7C100C3F394
S31508002FAC840301F01801013301EB501101FB0333C3
S31508002FBC14462B6087E700BF0C000020E8040020AD
S31508002FCC0014014088B108B5D0F8B43213B1002307
S31508002FDCC0F8B43209B1C0F8B0120123027080F8F7
S31508002FEC9C3203F0B1FE002008BD0220704700BFDA
S31508002FFC012210B50446D0F8B43280F89C225B68DE
S3150800300C01799847204603F003FF204603F0E4FEB7
S3150800301C002010BD19B1C0F8B41200207047022068
S3150800302C704700BF08B503F0E5FE002008BD00BFD9
S3150800303C08B5D0F8B4321BB11B68984700B908BD5F
S3150800304C022008BD08B5D0F8B4325B689847002052
S3150800305C08BD00BF38B5044600F52A75284600F0A9
S3150800306C57FB012094F8A812B4F8AE2201F01F03FE
S3150800307C8342C4F89402C4F8982215D00ED3022BB6
S3150800308C06D001F08001204603F0EEFE002038BD84
S3150800309C2946204600F0A6FA002038BD29462046C7
S315080030AC00F0F6F8002038BD2946204600F06EFAE6
S315080030BC002038BD70B5054641B9D0F89432032BBB
S315080030CC0FD0052B0C462ED0002070BDD0F8B4328C
S315080030DC9B69C3B190F89C22032A14D19847002007
S315080030EC70BD1646D0F86031D0F8642193420CD9DD
S315080030FC9B1A9A42C0F860318CBF9AB292B231468A
S3150800310C00F062FBE0E7022070BDD0F8B4321B6910
S3150800311C23B190F89C22032A00D19847284600F040
S3150800312C5BFB002070BDC5F8941203F09DFE20468B
S3150800313C70BD00BF70B5044681B91346D0F8942209
S3150800314C022A19D032F0040302D1802103F08CFE36
S3150800315C94F8A0320020012B0BD070BDD0F8B432F5
S3150800316C5B6963B390F89C22032A28D19847002000
S3150800317C70BD84F8A00270BDD0E90862964220D8CA
S3150800318CC369B3FBF2F502FB15350DB99A4226D97C
S3150800319CD4F8B432DB682BB194F89C22032A01D1FB
S315080031AC204698478021204603F05EFE204600F014
S315080031BC1FFB94F8A0320020012BCED1D9E70220B0
S315080031CC70BDB21A0D460262194692B200F0F4FAB4
S315080031DC2B462A462946204603F092FEB8E7D0F835
S315080031EC98229342D4D22A4600F0E6FAC4F89852AA
S315080031FCEEE700BF70B500224026044601251146AD
S3150800320C334603F013FE33468021C4F85851C4F8EC
S3150800321C64612046002203F009FE0021D4F8B83276
S3150800322CA561666284F89C52C4F894126160C4F86D
S3150800323CA41223B1D4F8B43220465B689847002010
S3150800324C70BD00BF01740020704700BF03460422FE
S3150800325C90F89C12002083F89D1283F89C227047E4
S3150800326C90F89C32042B04BF90F89D3280F89C325F
S3150800327C0020704790F89C22032A01D00020704742
S3150800328C08B5D0F8B432DB6903B19847002008BDFD
S3150800329C30B50B7883B003F06003202B0D4604463B
S315080032AC28D0402B26D053B18021204603F0DCFDD4
S315080032BC2046002103F0D8FD002003B030BD4B7822
S315080032CC092BF1D801A252F823F000BF5533000898
S315080032DC81330008B53200089D330008B532000862
S315080032ECA9330008E7330008B53200081D34000876
S315080032FC13330008D4F8B43229469B6820469847FD
S3150800330C002003B030BD89789F4D01292970CBD890
S3150800331C90F89C32022B00F00D81032B40F0FE80B6
S3150800332C002900F027814168012909D0C9B2FFF7A5
S3150800333C89FE297820466160FFF77AFE0228B3D009
S3150800334C204600F049FAB7E790F89C320322013B75
S3150800335C022BA9D8CB88022BA6D10121D0F8A432EE
S3150800336CC16003B1C260022204F10C01204600F0D0
S3150800337C15FAA1E790F89C32013B022B94D84B889E
S3150800338C012B99D10023C0F8A43200F025FA93E753
S3150800339C4B88012B90D1C0F8A432D1E78B88002B2F
S315080033AC82D1CB88002B7FF47FAF4D887F2D3FF6DB
S315080033BC7BAF90F89C32032B3FF476AFE9B280F8DA
S315080033CC9E1203F081FD204600F006FA002D00F04F
S315080033DCCD80022384F89C326EE700234A88ADF828
S315080033EC0630130A013B062B3FF65EAF01A151F8D6
S315080033FC23F000BFB53400089D340008C534000816
S3150800340CB5320008B5320008873400084334000882
S3150800341CCA88012A7FF448AF90F89C32002B3FF4F7
S3150800342C43AF022B40F29480032B7FF43DAF011D72
S3150800343C00F0B4F940E7037C002B7FF435AFD0F8E5
S3150800344CB4320DF106001B6B984707234370BDF881
S3150800345C0630EA886BB1002A3FF472AF934228BF54
S3150800346C134601461A462046ADF8063000F096F982
S3150800347CEA88002A7FF420AF62E7037C002B7FF4EE
S3150800348C13AFD0F8B4320DF106005B6B9847DEE744
S3150800349C027CD0F8B432002A61D19B6A0DF1060081
S315080034AC984702234370D2E7D0F8B0320DF10601E3
S315080034BC1B68007C9847CAE7D2B2052A3FF6F4AED9
S315080034CCDFE802F026201A140E03D0F8B0329B69F6
S315080034DC002B3FF4E9AE0DF10601207C9847B6E7C0
S315080034ECD0F8B0325B69002BF5D1DDE6D0F8B032F6
S315080034FC1B69002BEFD1D7E6D0F8B032DB68002B6E
S3150800350CE9D1D1E6D0F8B0329B68002BE3D1CBE6F3
S3150800351CD0F8B0325B68002BDDD1C5E6802103F00C
S3150800352CA3FC0021204603F09FFC29782046FFF7D0
S3150800353C89FDC1E600293FF403AF0121032341604D
S3150800354C80F89C32FFF774FD02287FF4F9AEABE6DF
S3150800355C0023014641F8083F00F020F9ACE6DB6A87
S3150800356C0DF1060098470223437070E7012384F88F
S3150800357C9C32A1E60223416080F89C32FFF762FD7B
S3150800358C204600F029F997E6EC04002038B50B78AC
S3150800359C0D4603F06003202B04460CD0402B0AD0B2
S315080035AC4BB18021204603F05FFC2046002103F036
S315080035BC5BFC002038BD94F89C32013B022BF0D8FA
S315080035CC2B79012BEDD8D4F8B43229469B682046C2
S315080035DC9847EB88002BECD10028EAD1204600F05E
S315080035ECFBF8E6E770B50B78044603F06003202B6E
S315080035FC0CD0402B0AD083B18021204603F034FC32
S3150800360C2046002103F030FC002070BDD4F8B432FB
S3150800361C20469B689847002070BD4B788A88012BFA
S3150800362CD5B23ED014D3032BE6D190F89C32022B9C
S3150800363C46D0032BE0D14B8833B96A0604D0CB8825
S3150800364C13B9294603F010FC204600F0C5F8DBE751
S3150800365C90F89C32022B3DD0032BCDD105F00F03ED
S3150800366C03EB8303120600EB830342D4D3F85831D9
S3150800367C002BC1D005F07F0303EB830600EB86060F
S3150800368C06F5AA7633B12946204603F009FC00282C
S3150800369C3BD00123336031462046022200F07EF8E7
S315080036ACB2E790F89C32022B0AD0032BA4D14B8894
S315080036BC002BA9D16E06C7D0294603F0E3FBC3E756
S315080036CC6B0699D0294603F0CFFB2046802103F0E0
S315080036DCCBFB99E768068FD1002311064CBF04F182
S315080036EC140104F5AA7120460B60022200F056F864
S315080036FC8AE79B69002B3FF47FAF05F07F035E1CBE
S3150800370C06EB860600EB8606BCE73060C3E700BF0F
S3150800371C0B7803704B784370CA788B7803EB0223CB
S3150800372C43804A790B7903EB02238380CA798B7918
S3150800373C03EB0223C380704710B50446802103F0BF
S3150800374C93FB2046BDE81040002103F08DBB00BF5B
S3150800375C00B3037830B4F3B10446002314F8015FC0
S3150800376C0133DBB2002DF9D15B000233032413803D
S3150800377C0B704C7004785CB1022300255A1CD2B22B
S3150800378CCC548D5410F8014F0233DBB2002CF5D112
S3150800379C30BC704770470223E8E700BF38B51346BC
S315080037AC02250A46C0E90733C0F89452002103F0F3
S315080037BC99FB002038BD00BF08B513460A46002100
S315080037CC03F090FB002008BD08B513460A460021F5
S315080037DC03F096FB002008BD08B504220023C0F8A8
S315080037EC942219461A4603F07DFB002008BD00BF3B
S315080037FC08B505220023C0F8942219461A4603F088
S3150800380C7FFB002008BD00BF72B6704762B67047D2
S3150800381CFFF7FABF10B500F0B9F900B910BDFCF7FF
S3150800382CA1FC0028FAD000F02DFCFCF7D3FE00F022
S3150800383CD1F900F0ADF9074B20F0604020F07F007D
S3150800384C986000F0A5F94468FFF7E0FF2346BDE849
S3150800385C1040184700ED00E072B170B5541EA4B2C2
S3150800386C0C440134461A0B784D1C8B5500F038FC69
S3150800387CA5422946F7D170BD704700BF2DE9F8431C
S3150800388C80460024FCF782FF08F1040906E0A359D8
S3150800389C0434AB4217D1B4F5007F1AD0D8F80060BF
S315080038AC59F80450A71900F01BFC2A463946002380
S315080038BC0220FCF7B7FF0028E9D00024FCF77AFFB2
S315080038CC2046BDE8F8830446FCF774FF2046BDE89D
S315080038DCF8830124F2E700BF70B50F4C0D46A042E1
S315080038EC15D00E4B99420CD123689D4207D0204621
S315080038FC294640F8045B4FF40072FFF7ADFF2046EB
S3150800390C70BD0646FFF7BAFF18B13446ECE7044C0F
S3150800391CEAE70446F3E700BFF40600200080000837
S3150800392CF00400202DE9F8430C46016824F4FF78CE
S3150800393C1D464B1C0746164628F0010833D0884509
S3150800394C26D10434641A3C4408F5007807F10409B6
S3150800395C05E016F8013B013D04F8013B15D000F0D3
S3150800396CBFFBA4EB0903B3F5007FF2D338464146F7
S3150800397CFFF7B2FF074600F1040988B14C4616F862
S3150800398C013B013D04F8013BE9D10120BDE8F88370
S3150800399C38464146FFF7A0FF074608B10168D0E74D
S315080039AC0020BDE8F883814649F8048B4146484611
S315080039BC4FF40072FFF750FF3968C0E74FF0FF333A
S315080039CC0249034A0B601360704700BFF0040020DD
S315080039DCF4060020104B30B44D1E1C1AA54213D801
S315080039EC0E4CA04210D9441E0C449C420CD820F410
S315080039FCFF730B4C23F00103A3420B46014606D07A
S31508003A0C30BC0848FFF78EBF002030BC704706480C
S31508003A1C30BCFFF787BF00BFFFFF0108FF7F000818
S31508003A2C00800008F0040020F4060020002330B5BE
S31508003A3C1F4C4D1E221A87B09542019332D820F49A
S31508003A4C7F721C4D22F00302AA422BD9451E0D4447
S31508003A5CA54227D80D18AD1AC5F30903C5F38F254A
S31508003A6C0BB10135ADB200240123049202940593DF
S31508003A7CFCF78CFE35B919E0049B954203F5806377
S31508003A8C049313D900F02CFB01A902A8FCF720FF1C
S31508003A9C0134A2B20028EFD00024FCF78BFE204696
S31508003AAC07B030BD1C46204607B030BD0124F4E7EC
S31508003ABCFFFF0108FF7F00080F490B68013318D078
S31508003ACCD1E9013010B5CC680344086923444C6924
S31508003ADC034488692344C969034482B00B4402AA87
S31508003AEC5B4242F8043D04210448FFF773FF02B019
S31508003AFC10BD0120704700BFF40600200C81000899
S31508003B0C0D4A0E4B0E4910681B6810B40C6803441A
S31508003B1C906823448C68034410311069234402F5D9
S31508003B2C84720968034412680B44D3420CBF012003
S31508003B3C002010BC704700BF0480000800800008F5
S31508003B4C088000080A4808B5036801330BD10948F0
S31508003B5C0368013305D0FFF791FE003018BF01202A
S31508003B6C08BD012008BDFFF789FE0028EFD108BD66
S31508003B7CF4060020F0040020004870470080000876
S31508003B8CFFF71CBFFFF726BFFFF750BFFFF7B8BFFD
S31508003B9CFFF7F2BF08B5FFF78FFF00B908BDBDE800
S31508003BAC0840FFF7CFBF00BF0022052010B4064B14
S31508003BBC064C07491A605A609A605C609A6010BC99
S31508003BCC18600A60704700BF10E000E03F1901005A
S31508003BDCF80800200022024B1A605A609A60704757
S31508003BEC10E000E0044B1B68DB0303D5034A13689B
S31508003BFC01331360704700BF10E000E0F80800209E
S31508003C0C044A054B12681868D20344BF0130186081
S31508003C1C704700BF10E000E0F8080020044A054B86
S31508003C2C12681868D20344BF01301860704700BF89
S31508003C3C10E000E0F8080020012838B504460D46C7
S31508003C4C04D94FF4DE710F4800F08CF904EB4404E8
S31508003C5C0D48E4000319597C1A7C914210D0DA6895
S31508003C6C1570DA68597C5D6801320131AA425974BB
S31508003C7CDA6003D902590120DA6038BD012038BD53
S31508003C8C002038BD3C7000083C090020012838B5D6
S31508003C9C04460D4604D94FF4EF710E4800F062F94C
S31508003CAC04EB44040C49E4000B19587C88B19A6857
S31508003CBC12782A70587CD3E901520132AA4200F1D3
S31508003CCCFF3058748CBF012001209A6084BF0A59B2
S31508003CDC9A6038BD3C7000083C09002070B5402538
S31508003CEC002201261B4B1C4803F118041B495C6176
S31508003CFC44195C604C190270DC6184191848C3E9D4
S31508003D0C02441C60174C02608819C3E908009861C4
S31508003D1CDA629A7483F82A601D821D850E70204615
S31508003D2C1149FFF74FF911492046FFF773F9204659
S31508003D3CFFF778F9D4F8C002FDF7A6FB00F054F9A2
S31508003D4CB0F5FA6F00D370BD4FF4FA60BDE8704059
S31508003D5C00F044B93C09002070090020B409002081
S31508003D6C6C090020F80900207400002010000020BF
S31508003D7C10B5054CD4F8C002FDF79AFB2046BDE8F1
S31508003D8C1040FFF735B900BFF80900203F29F8B5F0
S31508003D9C0D46044621D8134E29463078FFF74CFFBA
S31508003DAC012803D0B921104800F0DCF8ADB29DB15A
S31508003DBC013DADB20C4F2544013C00F091F914F8C5
S31508003DCC011F3078FFF738FF012803D0C221384687
S31508003DDC00F0C8F8AC42F0D1F8BDB521024800F0A5
S31508003DECC1F8D8E7700900203C7000082DE9F843A3
S31508003DFC1E4B1F4D0746D3F8C0028846FCF794FEA7
S31508003E0C2C785CB91B4B1C4E18783146FFF73EFFD5
S31508003E1C012823D000242046BDE8F883174E154BFD
S31508003E2C3178DFF85490013149441878FFF72EFFA2
S31508003E3C01280446EED1337899F800200133DBB219
S31508003E4C9A423370E6D109F101013846FFF704FDB1
S31508003E5C002233782A7088F80030DCE73378013B87
S31508003E6C3E2BD7D8054B28701C70D4E7F8090020D0
S31508003E7CFC0C0020B4090020BC0C0020FD0C002012
S31508003E8C2DE9F0411A4F82B03C78012C04D94FF435
S31508003E9CFF71184800F066F8174B04EB440403EB63
S31508003EACC404657C05B3402D28BF40250024134E59
S31508003EBCDFF840800DF107013878FFF7E7FE012897
S31508003ECC04D04FF4A171404600F04CF801349DF82B
S31508003EDC0730E4B2A54206F8013BEBD82B46074A55
S31508003EEC8121074802F0FEFF02B0BDE8F08100BF51
S31508003EFC700900203C7000083C090020FC080020D2
S31508003F0CF80900202DE9F041054602F051FE294634
S31508003F1C0446114803F002F880B298B1451EADB2BA
S31508003F2C0E4E0F4F2544013C14F8011F3078FFF74D
S31508003F3C83FE012804D04FF4B271384600F012F80B
S31508003F4CAC42F1D102F034FEBDE8F0410246402302
S31508003F5C0121014802F0D4BFF8090020B409002059
S31508003F6C3C70000808B500F0BBF8FCE710B500F08B
S31508003F7CADF8012806D000F01FF918B10C4C2378BF
S31508003F8C012B00D010BDFFF73BFE0A4B0A4A1B68F3
S31508003F9C1268134403F5FA739842F3D3002323707B
S31508003FAC00F012F90028EDD1BDE81040FFF732BC3D
S31508003FBC040D0020000D0020080D0020012208B574
S31508003FCC044B1A70FFF71CFE034B1860BDE808403B
S31508003FDCFFF7CCBF040D0020080D0020014B18601C
S31508003FEC704700BF000D0020014B1868704700BFD2
S31508003FFC000D002008B5FFF70BFC00F06FF8FFF773
S3150800400CD3FDFFF7BDFD00F0BDF800F013F8BDE8D1
S3150800401C0840FFF7D3BF00BF08B500F061F8FFF7FB
S3150800402CE1FD00F0CBF900F011F8BDE80840FFF708
S3150800403C9DBF00BF08B500F0FBFBFFF74FFE022241
S3150800404C014B1A7008BD00BF0D00002000B583B0E7
S3150800405C0DF107010948FFF7C9FE012802D003B084
S3150800406C5DF804FB0222064B9DF8071003481A70EC
S3150800407C00F0FAFB03B05DF804FB00BF0C0D002042
S3150800408C0D000020FFF774BE08B5074B1B78022BF2
S3150800409C03D0BDE8084000F0DFBBC9B2FFF776FED7
S315080040ACBDE8084000F0D8BB0D000020044B1B7877
S315080040BC032B9ABF034A32F813003F20704700BF00
S315080040CC0D00002078700008FFF7F0BF08B500F067
S315080040DCBBFB003018BF012008BD00BFFCF750B869
S315080040ECFCF752B8092802D93730C0B2704710B558
S315080040FC00F13003DCB202F041FF2346204442783B
S3150800410C02F00302022A08BFA4F12003D8B210BD9C
S3150800411C38B5054600090C46FFF7E4FF207005F094
S3150800412C0F00FFF7DFFF00236070A370204638BD31
S3150800413CF8B50027461E451C16F8014F02F01EFF5F
S3150800414C23462044417801F00301022908BFA4F153
S3150800415C2003DBB2A3F13002D2B2162AA3F13A013C
S3150800416C0DD806290BD9092A84BF373BDAB202EBDC
S3150800417C0713AE4203F0FF07DED13846F8BD002719
S3150800418C3846F8BD002310B5074C1A4607490848A7
S3150800419C237001F065FF00B910BD7721BDE810400A
S315080041AC0448FFF7DFBE00BFAC1100208070000882
S315080041BC540D002084700008024B1878B0FA80F071
S315080041CC40097047AC11002010B5FFF77FFF012896
S315080041DC02D0054C23780BB1002010BDFBF7D6FF97
S315080041EC0128F9D1207010BDAC11002038B5054650
S315080041FC047802F0C3FE23462044427802F00302F8
S3150800420C022A08BFA4F12003532B01D0032038BD82
S3150800421C02F0B4FE6B78184442785207F6D5312B67
S3150800422C05D0322B05D0332BF0D1022038BD002017
S3150800423C38BD012038BD00BF70B506460230FFF701
S3150800424C77FF0546043684B23046FFF771FF013C0A
S3150800425CA4B20544012CEDB206F10206F4D8304698
S3150800426CED43FFF765FFEDB2281AB0FA80F0400966
S3150800427C70BD00BFF8B5044616460D46002946D053
S3150800428C002844D02046FFF7B1FF032807463BD049
S3150800429C2046FFF7D1FF002800F08B80012F3CD079
S315080042AC65D3022F30D1A01CFFF742FF0746201D0D
S315080042BCFFF73EFF00062860A01DFFF739FF2B68A5
S315080042CC053F03EB0040286004F10800FFF730FFB8
S315080042DC2B683FB203EB0020286004F10A00FFF7B5
S315080042EC27FF2B6803442B607EB1002F0DDD0025BC
S315080042FC0C342046FFF71CFF6B1C70559DB2BD4253
S3150800430C04F10204F5DB00E000273846F8BD40F25C
S3150800431C63212948FFF726FEB4E7A01CFFF708FF20
S3150800432C0746201DFFF704FF00042860A01DFFF7B1
S3150800433CFFFE2B68043F03EB0020286004F10800FD
S3150800434CFFF7F6FE2B683FB203442B60002EDCD039
S3150800435C002FDADD00250A342046FFF7E9FE6B1C30
S3150800436C70559DB2BD4204F10204F5DBCDE7A01CE5
S3150800437CFFF7DEFE0746201DFFF7DAFE000228606F
S3150800438CA01DFFF7D5FE2B68033F03443FB22B60F5
S3150800439C002EBAD0002FB8DD002508342046FFF7CA
S315080043ACC7FE6B1C70559DB2BD4204F10204F5DBC9
S315080043BCABE74FF0FF37A8E7847000082DE9F84300
S315080043CCC14D2C782CB1012C05D0022C64D0032CB1
S315080043DC20D0BDE8F883FFF7D3FBFBF7F9FEBB4803
S315080043ECFBF72AFFBA48FBF727FFFBF7EDFE224639
S315080043FC0146B84801F062FE0646002800F0CB805C
S3150800440C0023B5482B70FBF717FF2046BDE8F84389
S3150800441CFBF708BFB14EB24F06F50C7238464FF48F
S3150800442C807102F083FA96F84192B9F1000F40F0C8
S3150800443CCF8070B107F5807207F5C0713846FFF763
S3150800444C19FFB0F1FF3F804600F02181002800F3E8
S3150800445CC280D6F84422D6F83C329A42B9D1A14841
S3150800446CFBF7EAFEFFF796FB0346002800F01F81D0
S3150800447C9D48FBF7E1FE9D48FBF7DEFE954802F0EA
S3150800448C09F99B48FBF7D8FE00232B70FBF7B4FE03
S3150800449CBDE8F843FFF7BEB9904E914F06F50C727E
S315080044AC38464FF4807102F041FA96F84182B8F119
S315080044BC000F7FD1A8B1424607F5C0713846FFF701
S315080044CCD9FEB0F1FF3F814600F0D380002808DD05
S315080044DC884CD7F880216368002B40F0C380C4E968
S315080044EC0020D6F84422D6F83C329A427FF471AFB3
S315080044FC0021784802F0E0F8002840F067817D4CEE
S3150800450C6368002B41D07848FBF796FE7A48FBF790
S3150800451C93FE636879491A467948A0FB0262D20869
S3150800452C01F10101F9D1764E0A70A6FB0302D208F5
S3150800453C02EB8200A3EB4003303301F8013D13462E
S3150800454C002AF2D16D48FBF777FE6E48FBF774FE2E
S3150800455C6A49E078FFF7DCFD6B49A078FFF7D8FDD0
S3150800456C6A496078FFF7D4FD69492078FFF7D0FDD2
S3150800457C6248FBF761FE6748FBF75EFED4E900016B
S3150800458CFFF702FB002800F02E815748FBF754FE74
S3150800459C03232B701DE75448FBF74EFE5E48FBF7CA
S315080045AC4BFE5E48FBF748FE0222524B2A70C3E9C3
S315080045BC00660EE7002348482B70FBF73DFE0220E9
S315080045CCFBF730FE06F50C70BDE8F84302F062B84E
S315080045DC00235348F0E75348FBF72EFE434647495A
S315080045EC474AA2FB0303DB0801F10101F9D1444652
S315080045FC43480B70A0FB0423DB0803EB8302A4EBF4
S3150800460C4202303201F8012D1C46002BF2D13B48F0
S3150800461CFBF712FE4448FBF70FFE384997F883015F
S3150800462CFFF776FD384997F88201FFF771FD374990
S3150800463C97F88101FFF76CFD354997F88001FFF76C
S3150800464C67FD2E48FBF7F8FD3248FBF7F5FD4146AA
S3150800465CD7F88001354AFFF795FAE0B12248FBF7FF
S3150800466CEBFDF6E621681944914263D10344636075
S3150800467C37E7194885F80080FBF7DEFD0320FBF7C2
S3150800468CD1FD06F50C70BDE8F84302F003B82848CE
S3150800469C85F80090F0E710482C70FBF7CDFD062046
S315080046ACFBF7C0FDBDE8F8430A4801F0F3BF0A481A
S315080046BC2B70FBF7C1FD0720FBF7B4FDBDE8F843EB
S315080046CC044801F0E7BF00BFAC110020B470000825
S315080046DCD8700008840F002000710008540D0020C3
S315080046ECB0110020FC710008087100081872000847
S315080046FC307200084C0D0020647100083413002039
S3150800470CCDCCCCCC707100083613002038130020A1
S3150800471C3A1300201472000810710008347100084E
S3150800472C8C710008D4710008E4710008B0120020DE
S3150800473CB07100083248FBF77FFD3248FBF77CFD69
S3150800474C636831491A463148A0FB02C2D20801F106
S3150800475C0101F9D1DFF8B4C00A70ACFB0302D20828
S3150800476C02EB8200A3EB4003303301F8013D1346FC
S3150800477C002AF2D12448FBF75FFD2548FBF75CFDC0
S3150800478C2149E078FFF7C4FC2249A078FFF7C0FC62
S3150800479C21496078FFF7BCFC20492078FFF7B8FC64
S315080047AC1948FBF749FD1E48FBF746FDD4E90001FD
S315080047BCFFF7EAF9B8B11248FBF73EFD1948FBF7C3
S315080047CC3BFDD7F88031C4E900398AE60023164840
S315080047DC2B70FBF731FD0420FBF724FDBDE8F843ED
S315080047EC124801F057BF00230F482B70FBF724FD26
S315080047FC0520FBF717FDBDE8F8430C4801F04ABF46
S3150800480C087100086471000834130020CDCCCCCC98
S3150800481C7071000836130020381300203A13002054
S3150800482C147200083471000800710008840F002007
S3150800483C0022044B9A6483F84220A3F844201A8079
S3150800484C9A70704774130020024B1878003018BF02
S3150800485C01207047741300200022024B83F8422073
S3150800486C704700BF74130020F8B50578FF2D41D0AA
S3150800487CB04C2378012B00D0F8BDC93D0646352D22
S3150800488C00F23C81DFE815F023013A013A018D006C
S3150800489C3A013A0105017A000D0114013A013A016F
S315080048AC3A013A013A013A013A013A013A013A0116
S315080048BC3A013A013A013A013A013A013A013A0106
S315080048CC3A013A013A013A013A013A013A013A01F6
S315080048DC3A013A013A013A013A013A019500B00017
S315080048ECBE00D2003A013A013A01DA003A01E9006F
S315080048FCF100FD00FFF760FCA8B9FE211022022387
S3150800490C8C4CE1702271A4F8443094F84230012B97
S3150800491C2CD0B4F844100123874884F84230BDE8FB
S3150800492CF840FFF7B1BB002310220126814C6371B6
S3150800493C22712680E570FFF7B9FBA071FFF7C4FB5F
S3150800494CE071FFF7C1FB0823D84020726672A67285
S3150800495CA4F84430FFF714F994F84230012B05D02B
S3150800496CB4F94410002987DD89B2D4E7FE22102356
S3150800497C0221E2702371A4F84410CCE7FFF796FBEA
S3150800498C73780138984235DDFF220123E270A4F8CA
S3150800499C44307178002940F0BE80FFF7FBF80028F8
S315080049ACDAD1FE2131220223E1702271A4F84430B7
S315080049BCABE7FF23E3704768A66C002F00F0B780BF
S315080049CC0025374416F8013B1D44FFF789FBB7420F
S315080049DCEDB2F7D1012100220823C4F80750A180B3
S315080049ECA271A4F8443090E7FFF760FB7378834212
S315080049FCC0F08C80FE2122220223E1702271A4F8D9
S31508004A0C443082E7FFF752FB72789042F2D9A16CD8
S31508004A1C4A48FEF721FFFF23E3707278A36C134410
S31508004A2CA36473780133A4F8443095E7FF23012275
S31508004A3CE3704368A4F84420A36466E70023FF25C3
S31508004A4C072008213E4AE57023716371A371C4F8E7
S31508004A5C0700A4F84410A26457E7FE21002202239B
S31508004A6CE1702271A4F844304FE70023FF20062199
S31508004A7C6278E0702371E3802372A4F844106271A3
S31508004A8C43E70021FF2201232180E270A4F8443079
S31508004A9C3BE7FEF7BFFEFF220123E270A4F8443081
S31508004AAC33E74168A06CFFF76FF80028F3D178E775
S31508004ABC0025FF232571E3706571FFF7F7FA0723C5
S31508004ACCA071E57125726572A4F844301DE7A56CD2
S31508004ADCFFF7ECFA721C411E2846FFF753F800281C
S31508004AEC3FF45FAFFF23E370FFF7E0FA0122A36CF4
S31508004AFC01380344A364A4F8442006E7FE212022C7
S31508004B0C0223E1702271A4F84430FEE671680B4862
S31508004B1CA16472787DE7B21CA06CFFF733F8002805
S31508004B2C3FF43FAF7278A36C1344A36414E73D4675
S31508004B3C50E700BF74130020771300207813002069
S31508004B4C5C72000830B40468ECB125781F2D0AD9BC
S31508004B5C3A2D18D0234602E03A2A08D00B465A7842
S31508004B6C591C1F2AF8D8002230BC1046704701344D
S31508004B7CA142A5F1300206D1302D04D130BC023346
S31508004B8C0360104670474FF0FF3230BC1046704732
S31508004B9CD8B110B5036882B004462BB11A781AB18D
S31508004BACD888A288904204D0002309200B6002B052
S31508004BBC10BD58780191FEF72FF810F001000199F5
S31508004BCCF2D123680B6002B010BD002309200B60DC
S31508004BDC704700BF01380A4411F8013B914200F8AE
S31508004BEC013FF9D1704700BFF8B5C56A00F1300727
S31508004BFC04462A46394640780123FEF763F8B0B9CD
S31508004C0C226AA369AA1A9A42E0700ED2A678012ED5
S31508004C1C01D80AE0A3691D44013E2A4601233946F8
S31508004C2C6078FEF74FF8012EF4D10020F8BD01206C
S31508004C3CF8BD00BF2DE9F843C378054663B92B7850
S31508004C4C032B10D0002268781146FEF7ABF800301B
S31508004C5C18BF0120BDE8F883FFF7C6FF0028F9D175
S31508004C6C2B78032BEED12B79012BEBD105F13001E7
S31508004C7C0B46002405F50C7203F8014B9A42FBD13E
S31508004C8C4FF0520C72204FF0AA0E612741264FF0B6
S31508004C9C55082B6985F814021A0A85F8183285F80E
S31508004CAC19224FEA13491A0EEB6885F81B221A0AC1
S31508004CBC85F81C3285F81D221A0C1B0E85F81F3236
S31508004CCCEB6985F81E225A1C85F8150285F81A9286
S31508004CDC85F82E82EA6285F82FE285F830C085F8C9
S31508004CEC31C085F8327085F8177285F8336085F807
S31508004CFC166201236878FDF7E5FF2C71A2E700BF61
S31508004D0C38B5C37804460D4613B1FFF76DFF68B97D
S31508004D1C2A46012304F130016078FDF787FF002845
S31508004D2C16BF4FF0FF3500200120E56238BD00BFE5
S31508004D3C4FF0FF330022994210B50446C270C36285
S31508004D4C2BD14AF6552294F82F1294F82E3243EAB0
S31508004D5C012393421FD1B4F8681094F8672094F88D
S31508004D6C663042EA012243EA0223104A23F07F43C3
S31508004D7C934218D0B4F8841094F8833094F88200CF
S31508004D8C43EA012340EA032020F07F40904214BFF7
S31508004D9C0220002010BD032010BDFFF7B1FF00282C
S31508004DACCFD0042010BD002010BD00BF46415400D2
S31508004DBC00232DE9F0410B6084B00F461546FFF72A
S31508004DCCC1FE061EC0F2DC80C24B53F82640002CEE
S31508004DDC00F003813C60237805F0FE057BB1607812
S31508004DECFDF71AFFC7070AD4002D00F0038110F04F
S31508004DFC040000F0C6800A2004B0BDE8F081002348
S31508004E0CF0B260702370FDF78BFDC60700F1BC800D
S31508004E1C0DB14507EFD400212046FFF789FF02287C
S31508004E2C00F0B680042800F0E380012800F2D18057
S31508004E3C002694F83C2094F83B3043EA0223B3F559
S31508004E4C007F40F0C68094F8472094F8463053EA21
S31508004E5C022309D1B4F8561094F8553094F8542016
S31508004E6C43EA012342EA032394F84020A361511E26
S31508004E7C0129A27000F2AD8094F83D1088B26081C9
S31508004E8C002800F0A680481E084240F0A28094F83C
S31508004E9C420094F8415045EA00252807258140F040
S31508004EAC988094F8447094F8430050EA072009D186
S31508004EBCB4F852C094F8517094F8500047EA0C278D
S31508004ECC40EA072094F83FC094F83E7057EA0C2C39
S31508004EDC7FD003FB02F20CEB15171744B84278D3B4
S31508004EECC01BB0FBF1F1002973D040F6F57E4FF6E6
S31508004EFCF57871458CBF4FF0020E4FF0010E414507
S31508004F0C0CEB0600374401F1020C75D994F85B10CA
S31508004F1C94F85A20C4F814C052EA0122C4E907606E
S31508004F2CA76256D1002D54D1B4F85E5094F85D00A2
S31508004F3C94F85C104FEA8C0240EA052002F2FF1244
S31508004F4C41EA0021B3EB522F616242D34FF0FF3294
S31508004F5C802194F8610094F86030226143EA0023BA
S31508004F6C012BE26021716AD04FF0030E5A4A84F87D
S31508004F7C00E01388002001339BB21380E38000E025
S31508004F8C0B2004B0BDE8F081032004B0BDE8F08125
S31508004F9C6D46294604F5FC7304F50E7613F8062CB3
S31508004FAC42B11F8813F8010C13F8022C40EA0720AB
S31508004FBC42EA00221033B34241F8042BEED105F134
S31508004FCC100755F8046B66B90320AF42F9D10428CB
S31508004FDC0ED00D2004B0BDE8F0810C2004B0BDE85D
S31508004FECF08131462046FFF7A3FE0128EDD820E7CD
S31508004FFC0120C6E72846C4E7C4F814C0C4E907600C
S3150800500CA762002DE5D00244BEF1020F626213D0EE
S3150800501C4FF0010E0CEB4C020CF0010C0CEB520C85
S3150800502C0CF2FF1CB3EB5C2FD3D34FF0FF3380226B
S3150800503CC4E90333227199E74FEA4C0CF0E7E36AAB
S3150800504C711C994204D02046FFF75AFE00288BD1D2
S3150800505C4AF65522002094F82F1294F82E32207115
S3150800506C43EA012393427FF47FAF618E94F8312093
S3150800507C94F8303042EA0122184943EA02238B425B
S3150800508C7FF472AFB4F8161294F8152294F8143209
S3150800509C42EA0122124943EA02238B427FF464AFA7
S315080050AC94F8192294F81D32B4F81A02B4F81E12A0
S315080050BC42EA002043EA012194F8182294F81C329B
S315080050CC42EA002243EA01234FF0030EC4E90332F5
S315080050DC4CE700BFC0130020C41300205252614194
S315080050EC7272416101292CD94269F8B59142074679
S315080050FC25D202780C46022A3DD0032A23D0012A4F
S3150800510C1DD1036A01EB5106D0F82CC003EB5621CE
S3150800511C61454CD1C6F30802013603EB56213A44D5
S3150800512C614592F830504AD1C6F30806BB1993F874
S3150800513C3000E30745EA002047D50009F8BD0120F1
S3150800514CF8BD01207047016AC36A01EBD411994274
S3150800515C28D1A10001F4FE7101F130033B445A88B1
S3150800516C39445B7891F8300043EA022340EA03207D
S3150800517C20F07040F8BD016AC36A01EB142199420C
S3150800518C05D0FFF7BDFD10B14FF0FF30F8BD61003B
S3150800519C01F4FF71394491F8313091F8300040EA46
S315080051AC0320F8BDFFF7ACFD0028D2D0ECE7FFF7DB
S315080051BCA7FD0028E8D13B6AD7F82CC0AAE73846E1
S315080051CCFFF79EFD0028AFD0DEE7C0F30B00F8BD55
S315080051DCB1F5001F29D2CA06F8B50C4623D1816849
S315080051EC05460461066819BB3378022B01D9736A24
S315080051FCEBB93389B3EB541F15D9736AAB61696183
S3150800520C8BB1C4F30802303603EB54241644C5E9B3
S3150800521C06460020F8BD7369023B8A1E9A421ED3C5
S3150800522C0023C5E905130220F8BD0220704719466C
S3150800523C77897F02BC42EED3304607E00128F2D9C3
S3150800524C73698342EFD9A742E6D82868FFF74AFF65
S3150800525C431C0146A4EB0704F0D10120F8BD738961
S3150800526CB06A02FB0303AB61C9E700BF2DE9F04145
S3150800527C03780446022B0D46164655D0032B32D01E
S3150800528C012B02D00220BDE8F081036A01EB51071D
S3150800529CC26A03EB572191425FD107F1010803EB70
S315080052AC5821EB07C7F3080763D50120274497F85D
S315080052BC30308A4203F00F0343EA061387F830307E
S315080052CCE07004D02046FFF71BFD0028DBD1C8F39D
S315080052DC0808C6F30716A044012388F83060E37063
S315080052EC0020BDE8F081016AC36A01EBD511994229
S315080052FC3AD10127AD0005F4FE7505F130012144BC
S3150800530C4B8826F070461A0402F070423243254444
S3150800531C85F83020100A130C120E48708B70CA7060
S3150800532CE7700020BDE8F081016AC36A01EB15211C
S3150800533C994203D0FFF7E4FC0028A4D101239D4031
S3150800534C05F4FF752544C6F3072285F8306085F801
S3150800535C3120E3700020BDE8F081FFF7D1FC00286E
S3150800536C91D1236AE26A98E7FFF7CAFC0028C0D0F5
S3150800537C89E7012327448A4287F83060E3700AD10B
S3150800538CC8F30808A04498F83030C6F3032223F073
S3150800539C0F061643A0E72046FFF7B2FC00287FF459
S315080053AC72AFEDE72DE9F04107468846066829BB3A
S315080053BCF5687369F5B901252C4606E0012815D060
S315080053CC013031D0AC4234D0736901349C4202D3DB
S315080053DC012D2ED9022421463868FFF783FE0028B2
S315080053ECECD1012C02D973699C4214D301242046B2
S315080053FCBDE8F0819D4228BF0125DDE73046FFF761
S3150800540C71FE01280446F1D9431C0DD073698342F9
S3150800541CEDD84546D0E74FF0FF3221463046FFF728
S3150800542C25FF50B10128E1D14FF0FF342046BDE8E5
S3150800543CF08100242046BDE8F081B8F1000F0CD0AD
S3150800544CB8F1010FD2D973699845CFD24146224695
S3150800545C3046FFF70BFF0028E4D1D6E90423023BBC
S3150800546C9A42F46001D2013A3261337943F001036E
S3150800547C3371BCE72DE9F84F8369CBB10569203543
S3150800548CB5F5001F14D2C5F3080688460446076806
S3150800549C3EB941690133836169B93B89B3EB551F41
S315080054AC29D930363E44E66125610020BDE8F88FDF
S315080054BC0420BDE8F88F7B89013B13EA5523F0D10C
S315080054CC3846FFF70FFE012881465CD9B0F1FF3F3D
S315080054DC19D07B69834218D9A0F10208023B4345CF
S315080054EC92BF00237B89BA6AC4F8149088BF08FB5C
S315080054FC0323A361D5E700230420A361D9E7384623
S3150800550CFFF772FB98B10120D3E7B8F1000FF2D080
S3150800551C61692046FFF746FF8146002835D00128E9
S3150800552C31D0B0F1FF3FEED0FB78002BE7D100224B
S3150800553C07F1300307F50C7103F8012B9942FBD1DF
S3150800554C7B69A9F102089A1E90452CBF0022BA6AFB
S3150800555C798938BF08FB0122FA62E9B14FF0000BD2
S3150800556C4FF0010A05E0FA6A7B8901325B45FA625B
S3150800557C0DD987F803A03846FFF736FB0BF1010B5C
S3150800558C0028F0D0BFE7022093E7072091E77B6954
S3150800559CA2EB0B02FA62A1E78B46F9E7416A2DE901
S315080055ACF0414B1C0446056806691AD14FF0E5080C
S315080055BC012704E000212046FFF75CFFB8B9A16972
S315080055CCEB6A994203D02846FFF79AFB78B9E36948
S315080055DC83F80080EF702369B342EBD30020BDE853
S315080055ECF081FFF7F5FD0028E0D0BDE8F08104282E
S315080055FC08BF0220BDE8F0812DE9F04F002187B0E5
S3150800560C05460768FFF7E4FD8246002847D14FF0A8
S3150800561CFF334FF0FF0B9846D9466B620CE00F2B05
S3150800562C41D04FF0FF09C5F8248000212846FFF722
S3150800563C21FF002840F0A380A969FB6A994205D08E
S3150800564C3846FFF75DFB002840F09980EC69267810
S3150800565C002E00F09980E27AE52E02F03F03AB713A
S3150800566CDFD01207DBD40F2B1DD0B9F1000F6AD08F
S3150800567C296ACB7ADB07D4D40846237810F80B2B87
S3150800568C01319B1A0134002BCBD111F8012B14F8DC
S3150800569C013B8842A3EB0203F5D1002BC1D150463E
S315080056AC07B0BDE8F08FAB6A002BBED070065BD591
S315080056BC2A6994F80DB006F0BF066A62627B5A45F1
S315080056CC54D1E17EA27E52EA01224FD101212278E1
S315080056DCCDE901B702F03F02013A02EB420002EBB8
S315080056EC8002CDE903A50596254693461C46DFF8A8
S315080056FCD8900B4613E0BBF1FE0F1DD8304601F0CF
S3150800570C85F9824634F81B0001F080F9824513D1DD
S3150800571C3346BB462B4A4A453CD019F8011F681834
S3150800572C40786E5C0BF1010746EA0026002BE2D1A5
S3150800573C4FF6FF729642EDD0DDE901B7DDE903A518
S3150800574C4FF0FF0971E7214604F10B0011F8012B04
S3150800575C4FEAC91343EA59099144884209F0FF09EB
S3150800576CF4D1CB4584D19AE7B145A7D00021284678
S3150800577C4FF0FF09FFF77EFE00283FF45DAF824627
S3150800578C504607B0BDE8F08F4FF0040A504607B0F4
S3150800579CBDE8F08F9C4623462C46DDE903A5217807
S315080057AC5A464906029F059EDDF804B006D5BCF19B
S315080057BC000F03D033F81230002BD7D1013E5FFA15
S315080057CC86F932E7F0720008E47200082DE9F04F0A
S315080057DCD0F820A08BB09AF80B3013F0A00840F044
S315080057ECF180D0F82890B9F80030002B00F07E81B3
S315080057FC4B4633F8022F08F10108002AF9D1044662
S3150800580C236807A80C2251460093FFF7E3F99DF885
S3150800581C2730DD0755D49B0740F1D180B44B08F1EE
S3150800582C0C08A3FB08384FEA980808F10108002170
S3150800583C20462768FFF7CCFC0546002840F0A980CF
S3150800584C064608E0ABB1002601212046FFF712FEFA
S3150800585C002840F09D80A169FB6A994205D038461C
S3150800586CFFF74EFA002840F09380E3691B78E52B86
S3150800587CE8D10136B045E7D1B8F10103019340F000
S3150800588CB180009BA169DB6A994240F0A080002197
S3150800589CE36903F1200203F8011B9342FBD10B22A7
S315080058ACD4E90701FFF796F9D4E907130122DB7A45
S315080058BC03F018030B73009BDA7028460BB0BDE88F
S315080058CCF08F002301278AF80B300B22A36207A955
S315080058DC5046FFF77FF93B46864E07220DF11B050E
S315080058EC03F00F0000F13001392988BF00F13701A8
S315080058FC1B0902F1FF3205F80119F1D17E200AA91C
S3150800590C114401F8140C002A4AD09AF800102029E0
S3150800591C08D0514603E011F8010F202802D00133B4
S3150800592C9A42F8D1591E5144072A0AA810448CBF2A
S3150800593C202010F8140C03F1010398BF0132072B31
S3150800594C01F8010FF0D92046FFF756FE054648BB6D
S3150800595C0137642F1FD00B2207A95046FFF73AF9D7
S3150800596C052F13D93B46A9F1020535F8022F002A53
S3150800597CB3D0102102F0010000EB4303D80348BF53
S3150800598C734001394FEA5202F4D1EEE73B46A4E7DD
S3150800599C0546042D91D1072528460BB0BDE8F08F96
S315080059AC1346BFE7042888D19DF827308AF80B30B0
S315080059BC9DF82730C4F828909B073FF52FAF4FF07A
S315080059CC010834E7062528460BB0BDE8F08F009889
S315080059DCFFF796F900283FF45AAF054628460BB050
S315080059ECBDE8F08F2169019B2046A1EB4311FFF717
S315080059FCEFFB0028F1D1216A024601F10B00D30115
S31508005A0C11F8016B43EA52033344814203F0FF0257
S31508005A1CF5D1DFF8E4B002920395009BA169DB6A25
S31508005A2C994204D00098FFF76BF90028D5D1E169A3
S31508005A3C029F0026D4F828804F734FF00F079DF865
S31508005A4C04A033460AF1FF3202EB420002EB800255
S31508005A5C012530460E73CF728E76CE764FF6FF79C9
S31508005A6C4FF0FF0E18E038F8123001324FEA132CBB
S31508005A7C4B5587F801C0BBBB0C2E21D84FF6FF73CC
S31508005A8C1BF80650023001F805E00D4485F801E0D4
S31508005A9C0C280ED81BF800504B4501EB050700F1F6
S31508005AAC0106E0D130460C2801F805E087F801E03C
S31508005ABCF0D94FF6FF70834202D038F812300BB982
S31508005ACC4AF0400A0123009A81F800A020460021DA
S31508005ADCD370FFF7CFFC00287FF47FAF019B013B07
S31508005AEC01939AD1039DCCE63046D1E7984686E6D3
S31508005AFC4FECC44E21100100E472000801293DD96F
S31508005B0CF8B504680D46636907468B422BD932BB38
S31508005B1C20461CE0012826D0411C31D0012D22D963
S31508005B2C63699D421FD2294600222046FFF79EFB39
S31508005B3CA0B923695A1C05D02279013342F0010217
S31508005B4C236122716369B34207D9354638682946F9
S31508005B5CFFF7C8FA06460028DCD10020F8BD012A52
S31508005B6C01D9934201D80220F8BD114620464FF0C0
S31508005B7CFF32FFF77BFB0028E8D0F8BD0220704700
S31508005B8C0120F8BD2DE9F04F0746D0F800B083B0D8
S31508005B9C0D4611F8013B2F2BFAD05C2BF8D00021BF
S31508005BACB96028781F2840F2198180B21F28BE6A6E
S31508005BBC2CD92F282AD05C2828D0A6F10209A84669
S31508005BCC01240EE029F8020F18F8010F631C1F2890
S31508005BDC1ED92F281CD05C281AD0B3F5807F11D07B
S31508005BEC1C46012100F0EEFE60B17F28EAD8222877
S31508005BFC08D02A238D4A03E012F8013F002BE1D086
S31508005C0C9842F9D1062003B0BDE8F08F0123002491
S31508005C1C2B441A781D462F2A03F10103F9D05C2A66
S31508005C2CF7D01F288CBF4FF000094FF004094CB170
S31508005C3C06EB440232F8023D202B01D02E2B07D15D
S31508005C4C013CF7D100230620338003B0BDE8F08F62
S31508005C5C002220213B6A26F8142003F10B0006EBE0
S31508005C6C440203F8011B8342FBD1B31E4FF0000814
S31508005C7C01E008F1010833F8020F2028F9D02E2884
S31508005C8CF7D0B8F1000F01D049F00309134633F8E1
S31508005C9C022D2E2A01D0013CF9D1002308229A465E
S31508005CAC08F1010838B320286CD02E286FD09342FF
S31508005CBC19D2A0456DD07F2878D82B2800F087807C
S31508005CCC2C21DFF870C1814200F081801CF8011F7D
S31508005CDC0029F8D1A0F14101192900F288804AF06F
S31508005CEC020AC0B276E00B2A00F09580A04552D085
S31508005CFC49F003094FD93B6A1978E52902D10521E0
S31508005D0C19703B6A082A04BF4FEA8A0A5FFA8AFAAC
S31508005D1C0AF00C020C2A46D00AF0030ABAF1030F51
S31508005D2C41D019F0020F08D1BAF1010F08BF49F09A
S31508005D3C1009042A08BF49F0080983F80B9038465D
S31508005D4CFFF75AFC3B6ADB7A00285AD15A073FF50B
S31508005D5C5AAFBB79DB065CD53B699BF80010C3F3DD
S31508005D6C080330335B44D87E9A7E032942EA002224
S31508005D7C05D1597D1B7D43EA012342EA0342BA60E9
S31508005D8C287812E749F0030936F8180088E7A04581
S31508005D9CF8D10B2A3FD04FEA8A0A5FFA8AFAA0464C
S31508005DAC0B220823F0E749F00209C6E70021CDE9E2
S31508005DBC003200F007FEDDE9003249F0020930B185
S31508005DCC1B49084410F8800C00287FF476AF5F2036
S31508005DDC49F00309396AC8540133D5E78022384695
S31508005DEC3B6ADA7203B0BDE8F04FFFF7F1B9A0F1E0
S31508005DFC6101192997BF2038C0B2C0B24AF0010A0E
S31508005E0CE8E704287FF4FFAE13F0040F08BF05205B
S31508005E1CF9E60520F7E63B6A49F003091A78E52AFC
S31508005E2C7FF476AF05221A703B6A71E7F5720008A3
S31508005E3C64720008017300082DE9F843436A814629
S31508005E4C01330E461ED0876A3888BD1CB0B16FF078
S31508005E5C130807F50077A8EB010801F1150406E00D
S31508005E6CBD420BD004F8010F35F8020B38B10021EE
S31508005E7C00F0A8FD08EB04030028F1D1002300224A
S31508005E8C33449A75D9F81C40002122464FF02E0847
S31508005E9C96F816C004F10B0712F8013B202B1DD0FF
S31508005EAC052BA2EB040508BFE523092D3AD070187B
S31508005EBC4372BCF1000F10D1A3F1410EBEF1190FBC
S31508005ECC0AD8092D34BF0825102594F80CE01EEACB
S31508005EDC050F1CBF2033DBB2837501319742DBD12A
S31508005EEC7018BCF1000F05D180F816C0237B002B67
S31508005EFC08BF304600234372E37A3372E18B627F24
S31508005F0C237F42EA012243EA02233360627E237E20
S31508005F1C43EA0223B380E27DA37D43EA0223F3809E
S31508005F2CBDE8F8837018BCF1000F01D180F8168013
S31508005F3C80F809800131BAE72DE9F84FFF270446A6
S31508005F4C05683E46042006E0FF2600212046FFF79A
S31508005F5C91FA002858D1A169002959D0EB6A8B42CD
S31508005F6C04D02846FEF7CCFE00284DD1E1690A7804
S31508005F7C002A48D0CB7AE52A03F03F03A371E3D075
S31508005F8C2E2AE1D023F020000828DDD00F2B44D18F
S31508005F9C500635D523694F7B02F0BF0663624B7BEF
S31508005FACBB42D1D1CA7E8B7E53EA0223CCD10122C5
S31508005FBC0878DFF8A8C000F03F00013800EB400372
S31508005FCC4FF6FF7A9646D4F8289000EB83000CF12E
S31508005FDC0C0809E0FE28B7D89E4629F8103001307F
S31508005FECE0452ED01CF8012F8B1893F801B08B5C6A
S31508005FFC43EA0B23BEF1000FECD15345F0D0A3E7CF
S3150800600CB242A1D1CBE704200023A361BDE8F88FE7
S3150800601C0028F9D10020BDE8F88F6EB901F10B0004
S3150800602C11F8012BF30143EA56061644814206F091
S3150800603CFF06F5D1BE42EDD04FF0FF330020636268
S3150800604CE4E70B785B0605D5FE283FF67DAF002303
S3150800605C29F81030013EF6B277E700BFE472000863
S3150800606C10B584B004AB43F8041D019018461446C9
S3150800607C0091FEF767FD021E14DB0F4951F822301A
S3150800608C0BB100201870019B3BB10020012C187035
S3150800609C41F8223009D004B010BD184641F8223018
S315080060AC04B010BD0B2004B010BD024601A9684609
S315080060BCFEF77EFE04B010BDC01300202DE9F0419A
S315080060CC92B0019170B3002302F01F0703600446D7
S315080060DC154603A93A4601A8FEF76AFE064618B104
S315080060EC304612B0BDE8F0810399654A04AB0791B6
S315080060FC07A801990F931192FFF744FD05F01C03AD
S3150800610CA8B90F9A92F90B20002AC0F2A1809DF823
S3150800611C2220A3B112F0110F17D16B0740F19A8008
S3150800612C0826DDE70926304612B0BDE8F0810BB12A
S3150800613C04280ED00646304612B0BDE8F081D306C8
S3150800614C05D4A8077CD5D1077AD50726C8E704262F
S3150800615CC6E707A8FFF73AFB47F008070028E9D176
S3150800616C0E9BDDF80CC000224821612020255974AD
S3150800617C9A73DA7318740E9B59769A75DA751876BB
S3150800618C0E9BDD720E9B9CF80020D97E9D7E032A01
S3150800619C45EA012505D1597D1A7D42EA012245EACF
S315080061AC024500229A76DA769CF80010032901D16A
S315080061BC1A755A75002201210E9B1A775A779A7707
S315080061CCDA778CF80310002D57D007A82946DCF887
S315080061DC2C80FFF793FC0028ACD1DDF80CC0013DF0
S315080061ECDCF82C3098453DD1CCF80C500E9B47F07A
S315080061FC2007C4E908839CF80010D87E9A7E0329E8
S3150800620C42EA002205D1587D197D41EA002142EA6D
S3150800621C01420021A260D88B5A7F1B7F27746174B8
S3150800622C42EA0022BCF8060043EA0223A080304664
S3150800623CE360C4F800C06161E16112B0BDE8F081A9
S3150800624CDDF80CC02A070E9BDCF82C80D1D5CEE7DE
S3150800625C062645E72D070E9BDDF80CC083D4DCF823
S3150800626C2C80C6E760464146FEF74AFDDDF80CC0B1
S3150800627CCCF80C5000287FF45DAFDCF82C80B5E721
S3150800628CC81300202DE9F04F9946002385B08A469D
S3150800629CC9F8003003A914460546FEF779FC804672
S315080062AC002839D195F81180B8F1000F34D12B7C20
S315080062BCD80773D56B69EF68FF1AA74228BF27461C
S315080062CC57B305F1280BC3F30801002946D10399E6
S315080062DC4A89013A12EA532257D0A8694B690238FF
S315080062EC023B984274D24B898E6A03FB0066002ED9
S315080062FC6ED07C0A164413D01019984288BF9C1A83
S3150800630C4878234632465146FCF790FC002848D07C
S3150800631C4FF0010885F81180404605B0BDE8F08FAE
S3150800632CEA69B24216D02B7C48785B060BD501235A
S3150800633C5946FCF7C7FC0028EAD12B7C039A23F0B4
S3150800634C40032B745078012332465946FCF76EFCF1
S3150800635C0028DDD16969EE61C1F30801C1F5007445
S3150800636CBC4228BF3C462831294422465046FEF7F3
S3150800637C31FC6B69D9F80020234422443F1B6B611E
S3150800638CA244C9F800209ED1C6E7D3B9A86801284B
S3150800639C1ED9411CBCD00399A8619FE74FF007088A
S315080063ACBAE72B7C5A060AD5E869801BA04206D2A6
S315080063BC0AEB40204FF400725946FEF70BFC6402B8
S315080063CCD7E7A96928680192FEF78CFE019ADEE7E1
S315080063DC4FF0020885F811809EE700BF2DE9F04FB3
S315080063EC9A46002385B08B46CAF8003003A9164690
S315080063FC0446FEF7CDFB8046002853D194F811804D
S3150800640CB8F1000F4ED1227C910740F18C8063695C
S3150800641CF34200D3DE43002E73D004F12802019216
S3150800642CC3F3080000284BD1039AB2F80A9009F175
S3150800643CFF3919EA53290FD1002B7DD1A068002802
S3150800644C00F08280012800F09D80421C26D0A368AB
S3150800645CA061039A03B9A060237C5B0655D4A7698F
S3150800646C5369023F023B9F4280F08C805389916AA4
S3150800647C03FB0717002F00F08580750A4F4415D0CB
S3150800648C09EB0501994288BFA3EB090550782B4601
S3150800649C3A465946FCF716FC002847D04FF0010837
S315080064AC84F81180404605B0BDE8F08FE369606951
S315080064BCBB4202D0E36883424ED8E761C0F30800BA
S315080064CCC0F50075B54228BF3546283020442A4603
S315080064DC5946FEF77FFB237C43F04003237463691C
S315080064ECE2682B449A4238BF1A461146DAF800205D
S315080064FC761B2A446361E160AB44CAF800208FD14D
S3150800650C227C42F020022274CCE750780123E269FF
S3150800651C0199FCF7D7FB0028C0D1237C039A23F0FA
S3150800652C400323749BE74FF00708BBE7E169C91BD7
S3150800653CA9421BD36D02D2E7A1692046FEF732FFAA
S3150800654C00287FF47FAFDBE749462046FEF72AFF93
S3150800655C00287FF477AFD3E7507801233A460199A0
S3150800656CFCF764FB002899D16069A6E70BEB41217F
S3150800657C4FF400720198FEF72DFB237C23F04003A1
S3150800658C2374D7E74FF0020884F811808AE700BF16
S3150800659C70B50A2982B00E4605461AD06C68002CCE
S315080065AC08DB2B1901343C2C1E7305DCAB686C60BC
S315080065BC0133AB6002B070BD01AB224605F10C018C
S315080065CC2868FFF70BFF019B1C1B18BF4FF0FF3405
S315080065DCECE70D21FFF7DCFFE0E700BFF0B583B071
S315080065EC01A90446FEF7D4FA002839D1237C9A0669
S315080065FC36D55B06019D3CD4216AEB6A994231D1AA
S3150800660C636ADA7A42F02002DA72A2682168C2F367
S3150800661C0720D8769A760978032903D1120C110A21
S3150800662C1A7559750021482061270126E2685876A3
S3150800663C4FEA122C1A7783F81DC04FEA124C120E29
S3150800664C997583F81EC0DA77D9759974D9741F763B
S3150800665C2846EE70FEF7EEFA237C23F0200323740B
S3150800666C03B0F0BD2846FEF74BFB0028F8D1019D78
S3150800667CC6E768780123E26904F12801FCF722FBD6
S3150800668C28B9237C019D23F040032374B4E7012029
S3150800669CE6E700BF10B582B00446FFF79FFF08B1C6
S315080066AC02B010BD01A92046FEF772FA0028F7D1F0
S315080066BC206002B010BD00BF2DE9F04182B00F4634
S315080066CC01A90446FEF764FA054600284DD1657CF7
S315080066DC002D4AD1E368BB4204D2227C12F0020F89
S315080066EC08BF1F46002263696261002F3DD0019ADC
S315080066FCB2F80A804FEA48283BB1013B7A1EB3FB35
S3150800670CF8F1B2FBF8F28A4257D2A668002E60D08E
S3150800671CA661002E30D16369C3F30802002A56D04D
S3150800672CE269B24253D0237C01995B06487804F19E
S3150800673C28070AD501233946FCF7C4FAC8B9237CBD
S3150800674C019A23F0400323745078394601233246C4
S3150800675CFCF76CFA68B96369E268E661934204D996
S3150800676C227CE36042F020032374284602B0BDE87D
S3150800677CF08101256574F8E7474513D84CE02046A7
S3150800678CFEF710FE064678B3721CF2D0012E1BD902
S3150800679C019B5B69B34217D96369B8454344A66143
S315080067AC636123D2237CA7EB080798073146E6D406
S315080067BC2068FEF797FC0646E6E7C8F10002134088
S315080067CC6361FF1AA669A4E702256574CDE7E2683A
S315080067DCC4E731462046FEF7E5FD01280646F3D008
S315080067EC431CC6D0A06093E7474663693B44C7F38E
S315080067FC0802636172B10199B01E4A69023A904265
S3150800680CE2D24E898A6A00FB0626002EDCD006EBFD
S3150800681C572681E716467FE76369E7E730B591B0F7
S3150800682C01900D46002205A901A8FEF7C1FA0446F7
S3150800683C10B1204611B030BD0E4A02AB019905A81D
S3150800684C0F920D93FFF79EF904460028F1D10D9B84
S3150800685C93F90B30002B0ADB002DEAD00B9BA8759D
S3150800686C002BE6D0294605A8FFF7E6FAE1E7062449
S3150800687CDFE700BFC813002030B59DB00190022297
S3150800688C02A901A8FEF794FA029B069308B11DB05B
S3150800689C30BD254A03AB06A8019910920E93FFF753
S315080068AC71F90028F3D10E9B93F90B30002B05DBFD
S315080068BC9DF81E30DA0703D50720E8E70620E6E739
S315080068CC029D0D9A2978D07E947E032944EA0024E9
S315080068DC0BD0DB0610D406A8FEF760FE0028D6D12E
S315080068ECD4B90298FEF7A6F9D1E7517D127D42EA92
S315080068FC012244EA0244ECE711A8002111951394ED
S3150800690CFEF766FC0028C2D111A8FFF715FB002874
S3150800691CD2D00428BBD1DEE70246214606A8FFF7EB
S3150800692CEDF80028DDD0B2E7C81300202DE9F041B8
S3150800693C804617460546002482B04E1EB44212DA2B
S3150800694C01AB012269463846FFF79CFC019B012BDB
S3150800695C09D19DF800300D2BF0D00A2B05F8013B18
S3150800696C04F10104EAD100239C4214BF40461846A0
S3150800697C2B7002B0BDE8F08110B50446002308461A
S3150800698C217894B0CDE901030393B1B101A8FFF7BF
S3150800699CFFFD14F8011F0029F8D1029A002A0EDB14
S315080069AC01986B4604A9FFF719FD40B9029A009B9A
S315080069BC9A4204D1039814B010BD0A46F1E74FF079
S315080069CCFF30F8E77F2819D989B910B40E4AC723BE
S315080069DC03E0802915D032F8023F98428CB201F1B7
S315080069EC0101F6D104F1800080B210BC7047FF2873
S315080069FC05D8054B803833F81000704770470020CF
S31508006A0C70470020F1E700BF08730008284AB0F564
S31508006A1C805F284B41F67D513CBF134661210433F8
S31508006A2C002943D0814241D870B433F8022C1E4653
S31508006A3CD4B26518A8424FEA122208DB04337AB19D
S31508006A4C33F8041C09B18142EFD970BC7047082A87
S31508006A5CFBD8DFE802F00F13191C1F2225280B00A0
S31508006A6C06EB440336F814100433EBE7A0F5E350B1
S31508006A7C80B2EAE7411A33F81100E6E7411A01F049
S31508006A8C0103C01A80B2E0E7103880B2DDE720387F
S31508006A9C80B2DAE7303880B2D7E71A3880B2D4E752
S31508006AAC083080B2D1E7503880B2CEE7704700BFC5
S31508006ABC08740008FC7500082023038000487047FA
S31508006ACC480000200A23038000487047680000200D
S31508006ADC08B590F89C32032B01D0002008BDFDF7B1
S31508006AECCFF9002008BD00BF08B5FDF7C9F900208D
S31508006AFC08BD00BF08B50846FDF704FA002008BD16
S31508006B0C10B50446812100F0A1F92046012100F0B8
S31508006B1C9DF9002010BD00BF10B504464023022283
S31508006B2C812100F083F9204640230222012100F03E
S31508006B3C7DF920464023034A012100F0E1F90020A3
S31508006B4C10BD00BF0819002010B50C7814F0600FA2
S31508006B5C07D14A7804460A2A05D00B2A14D0062AE5
S31508006B6C07D0002010BD01220E49FCF717FE0020A5
S31508006B7C10BD4A88120A212A0BD017220A49204628
S31508006B8CFCF70CFE002010BD8B7843B9054A136040
S31508006B9CE7E7CA880549172A28BF1722EFE7FCF743
S31508006BACCBFDDEE7C8150020510000205A00002056
S31508006BBC0048704708190020122301480B807047BB
S31508006BCC90000020042301480B807047A400002085
S31508006BDC30B40025013AD2B28C1C04EB4204020FE5
S31508006BEC092AD3B203F130028ABF37330A700B7005
S31508006BFC4D7002318C424FEA0010F0D130BC704710
S31508006C0C1A220B480B4B00681B680A80C01801D166
S31508006C1C0948704710B5094B08221C680849FFF744
S31508006C2CD7FF204604220749FFF7D2FF024810BDBA
S31508006C3CE8F7FF1FF0F7FF1FA8000020ECF7FF1F6F
S31508006C4CAA000020BA00002010B5044C0A460448D5
S31508006C5C2146FCF77DFD204610BD00BF48190020D3
S31508006C6CD876000810B5044C0A4604482146FCF7A9
S31508006C7C6FFD204610BD00BF48190020E8760008B5
S31508006C8C10B5044C0A4604482146FCF761FD20461B
S31508006C9C10BD00BF48190020B876000810B5044C82
S31508006CAC0A4604482146FCF753FD204610BD00BF92
S31508006CBC48190020C076000800F52C71D0F8E802B7
S31508006CCCFCF7C8B901EB810300EBC303D3F87C21AD
S31508006CDCD0F8E802FCF7EEB901EB810300EBC3032D
S31508006CECDA6BD0F8E802FCF725BA00BFD0F8E80250
S31508006CFCFCF7C0BA10B504460121D0F8E802FCF737
S31508006D0CA1FAD4F8E802BDE81040FCF773BA00BF44
S31508006D1C10B50446F9F722FAD4F8E802FCF796FA05
S31508006D2CA36923B1024A136943F00603136110BD24
S31508006D3C00ED00E008B5D0F8E802FCF791FABDE8DA
S31508006D4C0840F9F70DBA00BF38B5044600220825E5
S31508006D5C02211E4B1E48C3F8E8421860C4F8C0321C
S31508006D6C1846C3E90151C3E906221A62F9F716FE59
S31508006D7C20B14FF49F711748FDF7F4F80022182339
S31508006D8C1146D4F8C002FAF7D3FC58230022802106
S31508006D9CD4F8C002FAF7CCFCC02300228121D4F81F
S31508006DACC002FAF7C5FC4FF4887300220121D4F807
S31508006DBCC002FAF7BDFCD4F8C0024FF48073002267
S31508006DCC8221FAF7B5FC002038BD00BFF415002067
S31508006DDC005C00400077000808B5D0F8C002F9F747
S31508006DEC59FE032896BF024B0220185C08BD00BF4B
S31508006DFCFC76000808B5D0F8C002F9F761FE03283E
S31508006E0C96BF024B0220185C08BD00BFFC76000832
S31508006E1C08B5D0F8C002F9F76DFE032896BF024BE9
S31508006E2C0220185C08BD00BFFC76000810B51C468D
S31508006E3CD0F8C00213462246FAF764FB032896BF1D
S31508006E4C014B0220185C10BDFC76000808B5D0F87A
S31508006E5CC002FAF789FB032896BF024B0220185C7E
S31508006E6C08BD00BFFC76000808B5D0F8C002FAF7D2
S31508006E7CEBFB032896BF024B0220185C08BD00BF2B
S31508006E8CFC76000808B5D0F8C002FAF719FC0328F6
S31508006E9C96BF024B0220185C08BD00BFFC760008A2
S31508006EAC0B06D0F8C02206D401EB810102EBC10116
S31508006EBC91F86A01704701F07F03013303EB8303F2
S31508006ECC02EBC3039878704708B5D0F8C002FAF7F6
S31508006EDC05FB032896BF024B0220185C08BD00BFB1
S31508006EECFC76000808B5D0F8C002FAF78FFB032821
S31508006EFC96BF024B0220185C08BD00BFFC76000842
S31508006F0C08B5D0F8C002FAF75DFB032896BF024B0A
S31508006F1C0220185C08BD00BFFC760008D0F8C00239
S31508006F2CFAF76ABB012902D00020F9F70DB9084611
S31508006F3CF9F70AB970B500250C4E0D4CA41BA41014
S31508006F4CA54209D100F050F800250A4E0A4CA41B9C
S31508006F5CA410A54205D170BD56F8253098470135C1
S31508006F6CEEE756F8253098470135F2E730780008F1
S31508006F7C307800083078000834780008044B054A45
S31508006F8C1B681B6A002B08BF1346D3F8EC00704726
S31508006F9CC40000202801002082B001B901A942B121
S31508006FAC4BB113780B601278101C18BF012002B075
S31508006FBC70471046FBE76FF00100F8E703460244FA
S31508006FCC934200D1704703F8011BF9E749B1FF2A30
S31508006FDC8BBF8A230A700360012088BF4FF0FF30ED
S31508006FEC7047084670470000F8B500BFF8BC08BCE7
S31508006FFC9E467047F8B500BFF8BC08BC9E4670475D
S3150800700C2F626F6F746C6F672E74787400000000B3
S3150800701C2F64656D6F70726F675F6F6C696D6578DD
S3150800702C696E6F5F73746D33322E7372656300000D
S3150800703C433A2F576F726B2F736F6674776172654D
S3150800704C2F4F70656E424C542F5461726765742FBE
S3150800705C536F757263652F41524D434D335F5354CD
S3150800706C4D333246312F7573622E630000000800CB
S3150800707C3F000000303A0000433A2F576F726B2FCF
S3150800708C736F6674776172652F4F70656E424C54D8
S3150800709C2F5461726765742F536F757263652F660B
S315080070AC696C652E630000004669726D77617265BE
S315080070BC20757064617465207265717565737420CA
S315080070CC64657465637465640A0D00004F70656EBB
S315080070DC696E67206669726D776172652066696C80
S315080070EC6520666F722072656164696E672E2E2E36
S315080070FC000000004552524F520A0D004F4B0A0D24
S3150800710C000000005374617274696E6720746865B8
S3150800711C2070726F6772616D6D696E672073657129
S3150800712C75656E63650A0D0050617273696E67202A
S3150800713C6669726D776172652066696C6520746F15
S3150800714C2064657465637420657261736520626C6E
S3150800715C6F636B732E2E2E0045726173696E6720F2
S3150800716C000000002062797465732066726F6D20CA
S3150800717C6D656D6F7279206174203078000000009F
S3150800718C52656164696E67206C696E652066726FFC
S3150800719C6D2066696C652E2E2E4552524F520A0D7D
S315080071AC00000000496E76616C696420636865634B
S315080071BC6B73756D20666F756E642E2E2E45525246
S315080071CC4F520A0D0000000050726F6772616D6DA8
S315080071DC696E67200000000020627974657320745C
S315080071EC6F206D656D6F72792061742030780000A0
S315080071FC57726974696E672070726F6772616D2059
S3150800720C636865636B73756D2E2E2E00436C6F73F6
S3150800721C696E67206669726D776172652066696C3E
S3150800722C650A0D004669726D776172652075706422
S3150800723C617465207375636365737366756C6C79B5
S3150800724C20636F6D706C657465640A0D0000000030
S3150800725C4F70656E424C5400809A45418E418F8022
S3150800726C4545454949498E8F9092924F994F5555A8
S3150800727C59999A9B9C9D9E9F41494F55A5A5A6A792
S3150800728CA8A9AAABACADAEAFB0B1B2B3B4B5B6B7EC
S3150800729CB8B9BABBBCBDBEBFC0C1C2C3C4C5C6C7DC
S315080072ACC8C9CACBCCCDCECFD0D1D2D3D4D5D6D7CC
S315080072BCD8D9DADBDCDDDEDFE0E1E2E3E4E5E6E7BC
S315080072CCE8E9EAEBECEDEEEFF0F1F2F3F4F5F6F7AC
S315080072DCF8F9FAFBFCFDFEFF01030507090E10126F
S315080072EC1416181C1E000000222A3A3C3E3F7C7FCE
S315080072FC000000002B2C3B3D5B5D0000C700FC002A
S3150800730CE900E200E400E000E500E700EA00EB0033
S3150800731CE800EF00EE00EC00C400C500C900E6006A
S3150800732CC600F400F600F200FB00F900FF00D600D8
S3150800733CDC00A200A300A500A7209201E100ED0045
S3150800734CF300FA00F100D100AA00BA00BF0010231E
S3150800735CAC00BD00BC00A100AB00BB00912592257A
S3150800736C9325022524256125622556255525632551
S3150800737C512557255D255C255B25102514253425B7
S3150800738C2C251C2500253C255E255F255A255425CC
S3150800739C69256625602550256C256725682564258D
S315080073AC652559255825522553256B256A251825F3
S315080073BC0C25882584258C2590258025B103DF008E
S315080073CC9303C003A303C303B500C403A60398031E
S315080073DCA903B4031E22C603B50329226122B100F0
S315080073EC6522642220232123F7004822B0001922A3
S315080073FCB7001A227F20B200A025A00061001A034C
S3150800740CE0001703F8000703FF00010078010001EC
S3150800741C300132010601390110014A012E017901A8
S3150800742C060180014D00430281018201820184011B
S3150800743C840186018701870189018A018B018B01E9
S3150800744C8D018E018F019001910191019301940197
S3150800745CF60196019701980198013D029B019C0142
S3150800746C9D0120029F01A001A001A201A201A40175
S3150800747CA401A601A701A701A901AA01AB01AC01A8
S3150800748CAC01AE01AF01AF01B101B201B301B30159
S3150800749CB501B501B701B801B801BA01BB01BC0108
S315080074ACBC01BE01F701C001C101C201C301C4017F
S315080074BCC501C401C701C801C701CA01CB01CA016C
S315080074CCCD011001DD0101008E01DE011201F3016F
S315080074DC0300F101F401F401F8012801220212015A
S315080074EC3A020900652C3B023B023D02662C3F0220
S315080074FC40024102410246020A0153024000810140
S3150800750C8601550289018A0158028F015A02900197
S3150800751C5C025D025E025F029301610262029401E3
S3150800752C6402650266026702970196016A02622C7A
S3150800753C6C026D026E029C01700271029D0173024F
S3150800754C74029F0176027702780279027A027B022C
S3150800755C7C02642C7E027F02A60181028202A901AA
S3150800756C8402850286028702AE014402B101B20189
S3150800757C45028D028E028F0290029102B7017B039F
S3150800758C0300FD03FE03FF03AC0304008603880314
S3150800759C89038A03B1031103C2030200A303A303DD
S315080075ACC4030803CC0303008C038E038F03D80390
S315080075BC1801F2030A00F903F303F403F503F603BF
S315080075CCF703F703F903FA03FA033004200350040C
S315080075DC1007600422018A043601C1040E01CF0487
S315080075EC0100C004D0044401610526040000000013
S315080075FC7D1D0100632C001E9601A01E5A01001F5A
S3150800760C0806101F0606201F0806301F0806401F0E
S3150800761C0606511F0700591F521F5B1F541F5D1F7B
S3150800762C561F5F1F601F0806701F0E00BA1FBB1F70
S3150800763CC81FC91FCA1FCB1FDA1FDB1FF81FF91F6C
S3150800764CEA1FEB1FFA1FFB1F801F0806901F080670
S3150800765CA01F0806B01F0400B81FB91FB21FBC1F15
S3150800766CCC1F0100C31FD01F0206E01F0206E51F30
S3150800767C0100EC1FF21F0100FC1F4E2101003221F4
S3150800768C70211002842101008321D0241A05302C84
S3150800769C2F04602C0201672C0601752C0201802C24
S315080076AC6401002D260841FF1A0300004465666133
S315080076BC756C740057696E5553422042756C6B2075
S315080076CC496E746572666163650000004F70656E7D
S315080076DC424C5420557365720000000057696E556C
S315080076EC53422042756C6B204465766963650000CD
S315080076FC000201022E2E2F5553425F44455649432C
S3150800770C452F5461726765742F757362645F636F76
S3150800771C6E662E63000000004300504F5349580014
S3150800772C2E00002020202020202020202828282851
S3150800773C2820202020202020202020202020202027
S3150800774C2020208810101010101010101010101077
S3150800775C1010100404040404040404040410101087
S3150800776C1010101041414141414101010101010133
S3150800777C01010101010101010101010101011010C1
S3150800778C1010101042424242424202020202020207
S3150800779C0202020202020202020202020202101093
S315080077AC101020000000000000000000000000007F
S315080077BC00000000000000000000000000000000AF
S315080077CC000000000000000000000000000000009F
S315080077DC000000000000000000000000000000008F
S315080077EC000000000000000000000000000000007F
S315080077FC000000000000000000000000000000006F
S3150800780C000000000000000000000000000000005E
S3150800781C000000000000000000000000000000004E
S3090800782C000000004A
S30908007830310100080C
S309080078340D0100082C
S315080078380024F40001000000100000000104000004
S31508007848256B00080D6B0008556B00080000000042
S3150800785800000000F56A0008016B0008DD6A0008E8
S31508007868000000000000000000000000C56A0008CB
S3150800787800000000D16A000809022000010100C0C2
S31508007888320904000002FF000000070581024000D3
S31508007898FF070501024000FF0A0610010000004024
S315080078A801000000C56B0008D16B0008556C00087C
S315080078B8716C00080D6C00088D6C0008A96C00082E
S315080078C81201100100000040501DAC6000010102C1
S315080078D803010000040309041A030000000000005D
S315080078E80000000000000000000000000000000082
S315080078F800000000C800002000000000000000008A
S315080079080000000000000000000000000000000061
S315080079180000000000000000000000000000000051
S315080079280000000000000000000000000000000041
S315080079380000000000000000000000000000000031
S315080079480000000000000000000000000000000021
S3150800795800000000000000004300000000000000CE
S315080079680000000000000000000000000000000001
S3150800797800000000000000004300000000000000AE
S3150800798800000000000000000000000000000000E1
S31508007998000000000000000043000000000000008E
S315080079A800000000000000000000000000000000C1
S315080079B8000000000000000043000000000000006E
S315080079C800000000000000000000000000000000A1
S315080079D8000000000000000043000000000000004E
S315080079E80000000000000000000000000000000081
S315080079F8000000000000000043000000000000002E
S31508007A080000000000000000000000000000000060
S31508007A18000000000000000043000000000000000D
S31508007A280000000000000000000000000000000040
S31508007A380000000000000000D96F0008A56F0008C4
S31508007A48000000002E7700082C7700082D7700081C
S31508007A582D7700082D7700082D7700082D77000860
S31508007A682D7700082D7700082D7700082D77000850
S31508007A78FFFFFFFFFFFFFFFFFFFFFFFFFFFF0000FE
S31508007A880100415343494900000000000000000076
S31508007A9800000000000000000000000000000000D0
S31508007AA80000415343494900000000000000000057
S31508007AB800000000000000000000000000000000B0
S30908007AC800000000AC
S7050800059558
